:100000000C94500B0C9471400C94D1400C946D0BDB
:100010000C946D0B0C946D0B0C94DB400C946D0BDD
:100020000C946D0B0C94E5400C946D0B0C946D0BC3
:100030000C946D0B0C946D0B0C946D0B0C946D0B60
:100040000C944B410C946D0B0C946D0B0C946D0B3C
:100050000C9471410C9499410C94C8410C946D0B13
:100060000C946D0B0C946D0B0C946D0B0C946D0B30
:100070000C946D0B0C946D0B0C946D0B312E323275
:100080002E303500171515151515170012121212FE
:10009000121212001711111714141700171111174B
:1000A0001111170015151517111111001714141738
:1000B0001111170017141417151517000000000070
:1000C0000000000084008C0094009C00A400AC00A0
:1000D000B400BC004845414400474554202F00521D
:1000E00045424F4F540D0A0052455345540D0A00E6
:1000F0004A4A59004750530054532D4E5450303102
:100100005F585858585858006E74702E6A73742E81
:100110006D666565642E61642E6A70003030302E25
:100120003030302E3030302E303030003030302E05
:100130003030302E3030302E303030003030302EF5
:100140003030302E3030302E3030300008011C017D
:100150002C013C01F10611073107510730313233D0
:1001600034353637383941424344454600485454C3
:10017000502F312E312032303020485454500D0A47
:10018000436F6E6E656374696F6E3A20636C6F7354
:10019000650D0A436F6E74656E742D547970653AFF
:1001A00020746578742F68746D6C0D0A4361636800
:1001B000652D436F6E74726F6C3A206E6F2D6361A4
:1001C0006368650D0A436F6E74656E742D4C616EC5
:1001D00067756167653A20656E0D0A0D0A0048541F
:1001E00054502F312E3120323030204F4B0D0A43E6
:1001F0006F6E6E656374696F6E3A20636C6F7365C2
:100200000D0A436F6E74656E742D547970653A20D3
:10021000746578742F68746D6C0D0A43616368654A
:100220002D436F6E74726F6C3A206E6F2D63616335
:1002300068650D0A436F6E74656E742D4C616E6750
:10024000756167653A20656E0D0A0D0A3C21444FC1
:1002500043545950452048544D4C205055424C4928
:100260004320222D2F2F5733432F2F44544420480F
:10027000544D4C20342E3031205472616E736974A9
:10028000696F6E616C2F2F454E2220226874747046
:100290003A2F2F7777772E77332E6F72672F54523E
:1002A0002F68746D6C342F6C6F6F73652E6474647B
:1002B000223E3C48544D4C3E3C484541443E3C5413
:1002C00049544C453E54532D4E54502D534552568F
:1002D00045522053455455503C2F5449544C453EAB
:1002E0003C2F484541443E3C424F445920424743FD
:1002F0004F4C4F523D2223464646464646464622EE
:100300003E3C43454E5445523E3C423E00223E3C1C
:100310002F464F524D3E3C42523E3C464F4E54209B
:10032000434F4C4F523D22475245454E223E564187
:100330004C55452053415645443C2F464F4E543E64
:100340003C42523E00223E3C42523E3C42523E3CE7
:10035000494E50555420545950453D225355424D15
:100360004954222056414C55453D224150504C594C
:10037000223E3C2F464F524D3E004950004E4D000C
:10038000475700444E004243007A037D03800383B5
:100390000386032000240028002C00C0006401A86C
:1003A000C000FFFFFF0101A8C00101A8C0FF01A814
:1003B000C049502041444452455353005355424E86
:1003C0004554204D41534B00474154455741590036
:1003D000444E5320534552564552004144445245E1
:1003E000535300B103BC03C803D003DB034E3100F9
:1003F0004E32004E33004E3400ED03F003F303F6AB
:1004000003534552564552310053455256455232D8
:1004100000534552564552330053455256455234C7
:10042000000104090411041904400060008000A0C8
:100430000000504F574552204F4E004558544552EA
:100440004E414C2052455345540042524F574E2086
:100450004F55542052455345540057415443484446
:100460004F472054494D455220524553455400456D
:100470004E4332384A36302052454345495645208E
:100480004552524F5200415250205245515545530A
:10049000542054494D454F5554204552524F520017
:1004A00049434D50205041434B4554204348454318
:1004B0004B2053554D204552524F5200544350202B
:1004C0005041434B455420434845434B2053554DE1
:1004D000204552524F5200554450205041434B4505
:1004E0005420434845434B2053554D204552524FCD
:1004F000520049434D50204D455353414745004418
:100500004843502052454345495645204E414B28CB
:1005100052455452592900444843502052454E45B3
:1005200057414C20535441544500444843502052B5
:100530004542494E44205354415445004448435099
:100540002045585049524544205354415445004495
:100550004843502052454345495645205041434B5E
:100560004554204552524F52004E4254205245436A
:1005700045495645204552524F52004E425420465E
:100580004F524D4154204552524F52004E4254203A
:100590005041434B4554204552524F52004E425415
:1005A0002054494D45204F555428534552564552E5
:1005B0003129004E42542054494D45204F5554286E
:1005C0005345525645523229004E42542054494D0B
:1005D00045204F5554285345525645523329004E15
:1005E00042542054494D45204F55542853455256A6
:1005F0004552342900444E532054494D45204F550F
:100600005428534552564552312900444E532054E4
:10061000494D45204F55542853455256455232298D
:1006200000444E532054494D45204F5554285345BE
:1006300052564552332900444E532054494D4520CB
:100640004F5554285345525645523429004E545064
:1006500020554E53594E43524F4E495A4544004E31
:1006600054502054494D45204F5554285345525617
:1006700045523129004E54502054494D45204F5584
:1006800054285345525645523229004E5450205456
:10069000494D45204F55542853455256455233290C
:1006A000004E54502054494D45204F555428534531
:1006B000525645523429004E545020494C4C45471F
:1006C000414C20534552564552205245504C5900FA
:1006D0004E5450204C454150205345434F4E4420EA
:1006E00041444A5553540054494D4520494C4C45CA
:1006F00047414C00475053204E4D454120464F52F4
:100700004D4154204552524F52004E4D45412043D9
:100710004845434B53554D204552524F5200544982
:100720004D452044415441205245434549564520BA
:100730004552524F5200554E53594E432054494D45
:1007400045555000310432043B044A045A046F04F6
:100750008604A004BC04D704F204FF0417052A058C
:100760003C054F0569057B058C059D05B305C9054D
:10077000DF05F5050B06210637064D065F067506F3
:100780008B06A106B706D006E706F4060A071E0781
:1007900036076E772E636769006E732E6367690094
:1007A0006E622E63676900636C2E63676900656C17
:1007B0002E6367690073642E6367690066617669FA
:1007C000636F0092079907A007A707AE07B507BC9C
:1007D00007464958204E4554574F524B20534554D5
:1007E00054494E470054494D4520534552564552B1
:1007F0002053455454494E470054494D45205052CA
:100800004F564944452053455454494E4700544996
:100810004D452042524F414443415354204C4F4791
:10082000004556454E54204C4F47005359535445AC
:100830004D20494E464F4D4154494F4E00D107E59A
:1008400007F9070E0821082B084E54502041444A4E
:100850005553544D454E54204D4F44450042524F40
:100860004144434153542041444A5553544D454E0D
:1008700054204D4F4445004750532041444A55535E
:10088000544D454E54204D4F4445004A4A5920434B
:100890004C4F434B2041444A5553544D454E5420F0
:1008A0004D4F44450049085D0877088B084E4F209E
:1008B000414C41524D2854494D452053594E4352C5
:1008C0004F4E495A4544290054494D4520414C4119
:1008D000524D284E4F542053594E43524F4E495A71
:1008E0004544290054494D4520554E41444A5553ED
:1008F0005445440054494D45204F504552415449B8
:100900004F4E2054494D454F555400465552554E73
:100910004F20525443204D4F444500465552554EAA
:100920004F20475053204D4F444500555443204DD0
:100930004F44452856414C494429005554432050C2
:1009400050534F5554204D4F44452856414C49442F
:100950002900554E49564750532054494D45204E85
:100960004F2056414C4944004E4F2054494D45209C
:10097000494E50555400AD08C808E408F4080B0966
:100980001B092B093B095209680920485454502F70
:10099000003C2F413E3C42523E003F223E003C4242
:1009A000523E3C4120485245463D222E2F00545392
:1009B0002D4E54502D5345525645523C2F423E3CED
:1009C00042523E004243004954424C00223E3C42C7
:1009D000523E3C42523E494E54455256414C285399
:1009E00065632E2030206F72203E3635353334203B
:1009F00049676E6F7265293C42523E3C494E5055E4
:100A00005420545950453D225445585422204E41BB
:100A10004D453D224954424C222053495A453D22DE
:100A20003822204D41584C454E4754483D223522EE
:100A30002056414C55453D22003530223E3C2F5436
:100A4000483E3C54482057494454483D22313530B3
:100A5000223E54494D453C2F54483E3C5448205773
:100A6000494454483D22313530223E414D4F554E88
:100A7000543C2F54483E3C54482057494454483D28
:100A800022313530223E4E4F54453C2F54483E3C97
:100A90002F54523E003C2F54443E3C2F54523E00B3
:100AA0003C2F54443E3C54443E26656D73703B00DD
:100AB0003C2F54443E3C54443E42432041444A551A
:100AC0005354006D732E007365632C006F7665724E
:100AD0002039686F7572732E00444953545249424D
:100AE0005554494F4E002D2D2D2D2D3C2F54443E55
:100AF0003C54443E003C2F54443E3C54443E00266B
:100B0000656D73703B003C2F54443E3C54443E00A2
:100B10003C545220414C49474E3D2243454E54459A
:100B200052223E3C54443E004552525253540043DC
:100B30004C520050473D3100313530223E54494D32
:100B4000453C2F54483E3C54482057494454483D66
:100B500022353030223E4556454E543C2F54483EB7
:100B60003C2F54523E003C2F54443E3C2F54523EA6
:100B70000026656D73703B3C2F54443E3C54443E0C
:100B800026656D73703B002C44415441313A002C72
:100B9000434F44453A0028545950453A002C4E459D
:100BA00058543A002C434E543A00285354533A00B8
:100BB0003C2F54443E3C54443E002D2D2D2D2F2DD2
:100BC0002D2F2D2D202D2D3A2D2D3A2D2D003C543D
:100BD0005220414C49474E3D2243454E54455222F6
:100BE0003E3C54443E003C2F5441424C453E3C4226
:100BF000523E004F5045524154494E472054494DB2
:100C000045004D494E2E00484F555220004649524E
:100C10004D574152452056455253494F4E00454E7F
:100C20004332384A3630205245564953494F4E00D8
:100C30004D414320414444524553530054494D458E
:100C400020535441545553004F5045524154494F3D
:100C50004E204D4F4445004E455442494F53204E7F
:100C6000414D4500444E532053455256455200478E
:100C70004154455741592041444452455353005330
:100C800055424E4554204D41534B0049502041445C
:100C9000445245535300323030223E4954454D3C76
:100CA0002F54483E3C54482057494454483D223331
:100CB0003030223E56414C55453C2F54483E3C2F47
:100CC00054523E003C2F54443E3C2F54523E003C74
:100CD0002F54443E3C54443E003C545220414C4925
:100CE000474E3D2243454E544552223E3C54443EDD
:100CF00000222056414C55453D220022204D4158AE
:100D00004C454E4754483D2200222053495A453D08
:100D100022003C42523E3C494E50555420545950BA
:100D2000453D225445585422204E414D453D220018
:100D3000223E3C42523E003C42523E3C2F43454EF6
:100D40005445523E3C2F424F44593E3C2F48544D4F
:100D50004C3E003C42523E3C4120485245463D22DA
:100D60002E2F223E4D41494E204D454E553C2F41A0
:100D70003E3C42523E003C42523E003F455252529F
:100D80005354223E4552524F52204F46463C2F412B
:100D90003E3C42523E0026656D73703B3C4120480C
:100DA0005245463D22003F434C52223E4C4F472085
:100DB000434C4541523C2F413E003F50473D31227C
:100DC0003E5B325D3C2F413E26656D73703B3C417E
:100DD00020485245463D22003F50473D30223E5B71
:100DE000315D3C2F413E26656D73703B3C41204890
:100DF0005245463D22003C2F5441424C453E3C4228
:100E0000523E3C4120485245463D22003C2F423E46
:100E10003C42523E3C42523E3C5441424C452042B0
:100E20004F524445523D2231223E3C54523E3C54A6
:100E3000482057494454483D220022204D455448FB
:100E40004F443D22474554003C2F423E3C42523ED7
:100E50003C464F524D20414354494F4E3D22005392
:100E6000554E004D4F4E00545545005745440054D3
:100E70004855004652490053415400414955545287
:100E8000475550564E54532D4E54502D534552569F
:100E90004552303100454E4332384A3630205245B3
:100EA000563A00494E495449414C495A494E472EF9
:100EB0002E2E00494E495449414C495A4544004B55
:100EC0004559494E50555420494C4C4547414C00DA
:100ED0004D544B3333333920494E49542E2E2E0076
:100EE00043414C2052454D3A004448435020444928
:100EF0005341424C4544004448435020454E4142F2
:100F00004C4544004E545020525820454E41424CCE
:100F10004544004E54502052582044495341424CBD
:100F200045440042524F414443415354204C4F47A3
:100F3000004F5045524154494E472054494D4500B9
:100F4000475053204D4F4445205245414459004A93
:100F50004A59204D4F444520524541445900465579
:100F600052554E4F20475053204D4F444500554E4B
:100F7000495620475053204D4F444500454E43327B
:100F8000384A363020494E495445525200850E9514
:100F90000EA30EB30EBF0ED00EE00EE90EF70E0438
:100FA0000F130F230F310F400F4F0F5E0F6E0F7C8B
:100FB0000F56657273696F6E00504C454153452062
:100FC000434845434B204B455900504C4541534500
:100FD000205245534554004D41433A004448435044
:100FE000434E543A004E42432052454D3A00574139
:100FF000495420666F722054494D45205258004391
:101000004F4E4E4543542054532D4A4A59303200D6
:10101000434845434B204349524355495400504CA3
:1010200045415345205741495400434845434B20CF
:10103000434F4E4E4543544F5200B10FB90FCA0FA4
:10104000D70FDC0FE50FEE0FFF0F10101E102A1048
:1010500045585049524544200020524542494E448B
:10106000200052454E4557414C2000494E46494EBE
:10107000495459005010591062106B104A535400D3
:101080004B535400434354005554430050535400B1
:10109000484454007C108010841088108C109010EC
:1010A0002020202020202020202020202020202040
:1010B00000504F574552204F4E0045585445524E10
:1010C000414C2052455345540042524F574E204FF9
:1010D0005554205245534554005741544348444FBA
:1010E0004720524553455400454E43205243562015
:1010F0004552524F520041525020524551205449BE
:101100004D454F55540049434D502053554D2045B2
:1011100052524F52005443502053554D2045525285
:101120004F52005544502053554D204552524F5276
:101130000049434D50204D455353414745205243AC
:101140005600444843502052454345495645204E99
:10115000414B00444843502052454E4557414C00B6
:101160004448435020524542494E4400444843506D
:10117000204558504952454400444843502050436C
:1011800054204552524F52004E4254205243562052
:101190004552524F52004E425420464F524D4154F8
:1011A000204552524F52004E4254205041434B452D
:1011B00054204552524F52004E42542054494D45FE
:1011C0004F5554284E6F3129004E42542054494DFA
:1011D000454F5554284E6F3229004E4254205449F1
:1011E0004D454F5554284E6F3329004E42542054DC
:1011F000494D454F5554284E6F342900444E5320D5
:1012000054494D454F5554284E6F312900444E5393
:101210002054494D454F5554284E6F322900444EB5
:10122000532054494D454F5554284E6F332900449F
:101230004E532054494D454F5554284E6F34290084
:101240004E545020554E53594E43524F4E495A45D5
:10125000004E54502054494D454F5554284E6F313F
:1012600029004E54502054494D454F5554284E6F37
:101270003229004E54502054494D454F5554284E64
:101280006F3329004E54502054494D454F55542832
:101290004E6F3429004E545020494C4C4547414C28
:1012A000205245502E004E5450204C454150204174
:1012B000444A5553540054494D4520494C4C4547E8
:1012C000414C0047505320464F524D415420455207
:1012D000524F52004E4D45412043484B53554D20EF
:1012E0004552522E0054494D45204441544120520C
:1012F000435645525200554E53594E432054494D82
:1013000045555000A010B110BA10C910D910E810FE
:10131000F6100611151123113111421153116011EC
:101320006C11791188119611A711B811C911DA1130
:10133000EB11FC110D121E122F12401251126212EB
:10134000731284129512A612B612C312D412E512A9
:10135000F6122D2D2F2D2D202D2D3A2D2D3A2D2D00
:1013600000484F55522020204D494E2E002A2A3A3F
:101370002A2A3A2A2A002D2D3A2D2D3A2D2D0054B5
:10138000494D450D0A00444154450D0A0061646A07
:1013900075737465640076616C69640053545553C9
:1013A0000D0A00444353540D0A002D2D5A444100A8
:1013B00047505A4441002D2D524D43004750524D45
:1013C0004300504645432C475074707300504D54B1
:1013D0004B3030312C3331342C330024504D544BAE
:1013E0003331342C302C312C302C312C302C302C0F
:1013F000302C302C302C302C302C302C302C302C0D
:10140000302C302C302C312C302A32390D0A00246B
:10141000504D544B3331342C302C312C302C312C5A
:10142000302C302C302C302C302C302C302C302CDC
:10143000302C302C302C302C302C302C302A3238C0
:101440000D0A004649582049502041444452455312
:101450005300464958205355424E4554204D415360
:101460004B004649582044464C5420474154455768
:1014700041590046495820444E5320534552564541
:10148000520044484350205553452F554E5553451F
:1014900000424C4F41444341535420414444522E56
:1014A00000424C4F41444341535420494E54564C02
:1014B0000042434153542043414C20524543562E51
:1014C0000054494D45205A4F4E4500475053204E39
:1014D0004F444154412054494D45520047505320F8
:1014E000554E53594E432054494D4552004E4D459B
:1014F000412053454E54454E5345003150505320E2
:10150000494E5055542045444745004E54502052B2
:10151000582054494D454F55540041444A55535461
:10152000205749445448005155495420544F204DA8
:1015300041494E00431452146214731482149114DE
:10154000A114B114C114CB14DC14ED14FB140B154D
:101550001A1527154A5354285554432B393A30301D
:1015600029004B5354285554432B393A3030290025
:10157000434354285554432B383A303029005554AE
:10158000432855544320303A3030290050535428D2
:101590005554432D383A3030290048445428555486
:1015A000432D393A303029005415621570157E15D7
:1015B0008C159A15907E0000907E000080700000CF
:1015C00000000000808FFFFF7081FFFF46555255DD
:1015D0004E4F282447507470732900554E49562E9B
:1015E00028244750524D432900554E49562E282451
:1015F00047505A44412900CC15DB15E91546414CAA
:101600004C204544474500524953452045444745F1
:1016100000FD15071644495341424C4500454E41D3
:10162000424C450015161D1644495341424C450095
:10163000454E41424C45284E5450204D4F4445297B
:10164000002816301657494454483A2020202020BC
:101650007365630054494D454F55543A202020206E
:10166000206D7300544F55543A202020202073657C
:101670006300544F55543A202020202073656300A6
:10168000494E54455256414C3A20202020207300A8
:101690002F3136002D2D204D454E55202D2D00008B
:1016A00011241FBECFEFD0E1DEBFCDBF12E0A0E01E
:1016B000B1E0E4E1F6EC02C005900D92AA3BB1075F
:1016C000D9F71BE0AAEBB2E001C01D92A53AB10721
:1016D000E1F70E949F0E0C9408630C940000809127
:1016E0007C01882359F4809167099091680990934F
:1016F000880B8093870B81E080937C010895A0E2A2
:10170000B0E0E5E8FBE00C949D610E94831982E063
:101710000E948C4B01C0A895F999FDCF8EE090E016
:1017200060E570E00E94036301C0A895F999FDCFC0
:101730008CE090E06AE070E80E94036301C0A89525
:10174000F999FDCF80E290E044E651E068EA70EC60
:101750000E94FB6201C0A895F999FDCF84E290E058
:1017600040E05FEF6FEF7FEF0E94FB6201C0A89542
:10177000F999FDCF88E290E041E051E068EA70EC31
:101780000E94FB6201C0A895F999FDCF8CE290E020
:1017900041E051E068EA70EC0E94FB62CE010196E4
:1017A00068EF70E00E94F66101C0A895F999FDCF3D
:1017B000CE01019660E170E040E150E00E94E362FA
:1017C00001C0A895F999FDCF8E010F5F1F4FC80189
:1017D00068E071E00E94F661C80160E470E040E2F8
:1017E00050E00E94E36201C0A895F999FDCF8E01F7
:1017F0000F5F1F4FC8016CE171E00E94F661C801E4
:1018000060E670E040E250E00E94E36201C0A8950B
:10181000F999FDCF8E010F5F1F4FC8016CE271E097
:101820000E94F661C80160E870E040E250E00E946A
:10183000E36201C0A895F999FDCF8E010F5F1F4F9C
:10184000C8016CE371E00E94F661C80160EA70E0D3
:1018500040E250E00E94E36201C0A895F999FDCFF3
:1018600080EC90E04FEF51E068EA70EC0E94FB6280
:1018700001C0A895F999FDCF84EC90E060E070E09C
:101880000E94036301C0A895F999FDCF86EC90E012
:1018900060ED77E00E94036301C0A895F999FDCF40
:1018A00088EC90E068E873E10E94036301C0A895AA
:1018B000F999FDCF8CE390E061E070E00E94036352
:1018C00001C0A895F999FDCF8CEC90E060E070E044
:1018D0000E94036301C0A895F999FDCF80ED90E0C7
:1018E00064EB70E00E94036301C0A895F999FDCFF5
:1018F00082ED90E064E873E00E94036301C0A89564
:10190000F999FDCF8EE390E065EA73EC0E940363E2
:10191000A096E4E00C94B9610F931F930E94E91C18
:1019200083B180958F70873069F40E947F0B0E948D
:10193000831983E00E948C4B82E00E947F4BA89524
:10194000FECFA895F999FDCF8EE390E00E94A962A1
:10195000855A934C21F00E947F0B01C0A895F999FC
:10196000FDCF8EE090E00E94A9629093E404809302
:10197000E30401978E5F9F4F40F080E590E09093E5
:10198000E4048093E30401C0A895F999FDCF8CE0AD
:1019900090E00E94A9629C019F779093D307809367
:1019A000D207C90101978E5F9F4F50F084E1809369
:1019B000D5078CE390E09093D3078093D20710C0B3
:1019C00037FF0CC080916B0990916C09019711F061
:1019D00084E101C085E18093D50702C01092D5074C
:1019E0008091D507882309F040C080E290E044E66A
:1019F00051E068EA70EC0E94981B6093AA0470930F
:101A0000AB048093AC049093AD0484E290E040E09A
:101A10005FEF6FEF7FEF0E94981B6093AE047093AF
:101A2000AF048093B0049093B10488E290E041E069
:101A300051E068EA70EC0E94981B6093B2047093C6
:101A4000B3048093B4049093B5048CE290E041E039
:101A500051E068EA70EC0E94981B60935E097093F5
:101A60005F09809360099093610980E190E06EE4E2
:101A700079E048EF50E00E94751B8091030167E513
:101A800079E00E94543B8091040169E579E00E946D
:101A9000543B809105016BE579E00E94543B80ED59
:101AA00090E00E94A9622FEF8F3F920711F484EB20
:101AB00090E0909366098093650982ED90E00E9422
:101AC000A9624FEF8F3F940711F484E893E090935D
:101AD00068098093670980E490E061EF76E048E070
:101AE00051E00E94521B80E690E061E177E04CE11A
:101AF00051E00E94521B80E890E061E377E04CE205
:101B000051E00E94521B80EA90E061E577E04CE3EF
:101B100051E00E94521B80EC90E04FEF51E068EAE8
:101B200070EC0E94981B60937707709378078093FE
:101B3000790790937A0701C0A895F999FDCF84ECB5
:101B400090E00E94A96290939807809397078F5F17
:101B50009F4F31F4109298071092970701C0A895F3
:101B6000F999FDCF86EC90E00E94A96290939607C8
:101B70008093950701978E5F9F4F40F080ED97E02F
:101B8000909396078093950701C0A895F999FDCF8A
:101B900088EC90E00E94A96290939D0780939C0737
:101BA0008F5F9F4F31F488E893E190939D07809376
:101BB0009C0710916409012F077011F011C0A895BE
:101BC000F999FDCF8AEC90E00E94A96297FD08C0C8
:101BD00080FF06C0187F11601093640901C0A895AA
:101BE000F999FDCF8CE390E00E94A9624FEF8F3FFF
:101BF000940711F480E090E00230E1F42091640950
:101C0000277C20936409AC01477050704130510526
:101C100011F4286004C04230510519F4206120936A
:101C2000640983FF07C0809164098064809364091C
:101C300001C0A895F999FDCF8CEC90E00E94A962B3
:101C4000809372098F3F21F41092720901C0A89508
:101C5000F999FDCF80917209E82FF0E0EE0FFF1F98
:101C6000EE0FFF1FEC54FA4E85919591A591B4911A
:101C70008093770190937801A0937901B0937A01D2
:101C80001F910F910895EF92FF920F931F93E09091
:101C90009707F090980700E010E083E591E06DE190
:101CA00071E00E94813EE61AF70A080B190BB70192
:101CB000C8011F910F91FF90EF900895EF92FF924E
:101CC0000F931F93E0909907F0909A070027F7FC75
:101CD0000095102F81E491E06DE171E00E94813E5A
:101CE000E61AF70A080B190BB701C8011F910F91EB
:101CF000FF90EF9008950F931F938C010E94733D06
:101D0000005110406F717070060F171F10939A07E3
:101D1000009399070C33110534F48CE390E0909311
:101D20009A0780939907A1E4B1E0EDE1F1E082E147
:101D300001900D928150E1F71F910F910895A4E059
:101D4000B0E0E5EAFEE00C948F61F8941092680030
:101D50001CBA1DBA89E88093640080E885BF85BFFE
:101D600080BF9FEF92B980E185B918B813E01BB925
:101D700091B980EB84B98FE787B982EC8AB988E0A2
:101D800090E00E94A36260939E0770939F078093E8
:101D9000A0079093A10789B18073803129F411982D
:101DA00082E08093640905C0803239F41298109360
:101DB000640989E080937D0103C010981092640942
:101DC00080E18CBD81E08DBD16BC22E024BD83E0A6
:101DD00085BD97EC97BD20936E001092B2002093C2
:101DE000B00084E08093B1009093B3002093700022
:101DF0008091640987708250823080F485EA90E097
:101E00009093C5008093C4002093C00086E0809327
:101E1000C20088E98093C1008091C60084B780FF2A
:101E200004C081E00E94554F13C081FF02C082E0D0
:101E300007C082FF02C083E003C083FF09C084E0C3
:101E40000E94554F81E090E090936C0980936B095C
:101E500014BE8CE028E130E00FB6F894A8952093EA
:101E600060000FBE8093600078940E94021A0E9466
:101E70008C0C80E58CBD5E9A80E190E00E94551A42
:101E80000E942615882381F484E162EA7AE00E94A8
:101E900055140E94831981E10E948C4B88E00E94B6
:101EA0007F4B1798A895FECF0E94FC170E948319BC
:101EB00080E00E948C4B80E00E947F4B88E061E0D4
:101EC0004CE750E00E94B419C090640927E0C22298
:101ED0000E945C1A8C010CC0A89582E0C81619F407
:101EE0000E94CE5305C093E0C91611F40E94B2506F
:101EF0000E945C1A801B910B805D974068F30E94E2
:101F0000831983E0C81631F48EE00E948C4B87E081
:101F10000E947F4B8091640987FF0BC085E00E947F
:101F20008C4B89E00E947F4B8091640988730E94EA
:101F300048528091D5078823F1F081E090E090939A
:101F4000D7078093D607A8E0B1E0EDE1F1E082E1A8
:101F500001900D928150E1F78091D507843119F4F9
:101F60000E94BD2703C086E10E949B28882339F088
:101F70000E94554F04C01092D7071092D60792E0E6
:101F8000C91649F48091640986FF02C083E007C046
:101F9000C092690006C023E0C21631F482E080934B
:101FA00069001CBA81E08DBB10926C0910926B091C
:101FB0000E945C1A2C013E010894611C711C50ECBB
:101FC000352E46E0242EA8950E949621823019F4E1
:101FD0000E94022009C0833019F40E94762604C0B2
:101FE000843059F50E94E323182F0E94AF15112366
:101FF00021F18091640990E087709070892BD1F471
:10200000163091F4809173098823A1F0A1E4B1E026
:10201000EDE1F1E082E101900D928150E1F7109243
:102020004B091092730906C01B3121F480E490E043
:102030000E947B0E812F0E94554F82E0C81619F432
:102040000E94CE5305C093E0C91611F40E94B2500D
:10205000F894A090830BB090840B1092840B109294
:10206000830B8090850B9090860B1092860B1092BC
:10207000850B789421E0A216B10429F081E088163E
:10208000910409F0F9C1F89480917F0B9091800B35
:10209000A091810BB091820B89839A83AB83BC831F
:1020A0007894C3010E949C1D009721F43092060190
:1020B00081E0AEC0AFE2B1E0FC0182E101900D929F
:1020C0008150E1F780910601803461F580918F0B9A
:1020D0008823F9F48091330190913401892BC9F45C
:1020E0008091310190913201892B99F480912F01D7
:1020F00090913001892B69F489819A81AB81BC81EF
:102100000197A109B10989839A83AB83BC8382E0DB
:1021100043C080918F0B823009F053C081E08093DF
:102120008F0B4FC0803809F04CC080918F0B8823F3
:1021300009F047C08091330190913401479709F02D
:1021400040C08091310190913201CB97D1F58091BF
:102150002F0190913001CB97A1F589819A81AB81B4
:10216000BC810196A11DB11D89839A83AB83BC8379
:1021700080917F0B9091800BA091810BB091820B8D
:102180000196A11DB11D80937F0B9093800BA093AE
:10219000810BB093820B81E080938F0BC3010E946F
:1021A0009C1DAFE2B1E0FC0122E101900D922150B3
:1021B000E1F7892B31F4309206011092860B1092D0
:1021C000850B89819A81AB81BC8120917701309107
:1021D00078014091790150917A01820F931FA41FD9
:1021E000B51F89839A83AB83BC83C3010E949C1D66
:1021F000ADE1B1E0FC0182E101900D928150E1F787
:1022000080918F0B813039F41092060110928F0B60
:1022100080937D010AC080918F0B823031F48CE372
:1022200090E090931E0180931D0191E0A916B104E6
:1022300009F0CEC00E94F51D0E94C82F0E949E2961
:102240008091970790919807892B61F1809174098B
:10225000909175090197E1F40E94430E7B018C0176
:1022600016161706180619064CF10E94AB32882381
:1022700011F00E94554FA3E5B1E0EDE1F1E082E1FC
:1022800001900D928150E1F782E00E94EC4F16C060
:10229000A3E5B1E0EDE1F1E082E101900D92815022
:1022A000E1F709C0A3E5B1E0EDE1F1E082E10190E1
:1022B0000D928150E1F7EE24FF248701D09064094C
:1022C00027E0D22280917309882361F5DD20B1F4E3
:1022D0000E945E0EAB01BC01141615061606170609
:1022E0002CF18091AA049091AB04A091AC04B09120
:1022F000AD040097A105B105C9F010C083E0D81660
:1023000089F48091910B882369F40E945E0EAB01E1
:10231000BC01141615061606170644F081E08093DA
:10232000730904C040E050E060E070E08091710902
:102330008F5F809371098C33A9F410927109809199
:102340006D0990916E09A0916F09B0917009019685
:10235000A11DB11D80936D0990936E09A0936F0923
:10236000B093700980916209882319F40E94794D15
:102370002FC0843019F40E94554C2AC0853021F5B5
:1023800092E0D91641F021E0D21629F0809173092C
:10239000882309F4DFC180E00E94784B8091970781
:1023A00090919807892B61F080917409909175093B
:1023B000019731F481E0B801A7010E940B4C08C0DD
:1023C00081E00E94784B04C0863011F40E94994B42
:1023D00081E08816910409F04FC0809164098770EC
:1023E00029F410927D0110927C010BC0833049F0DA
:1023F000813069F50E94EC4F10927D0110927C01B2
:1024000026C08091990790919A0720917C092130EC
:1024100019F4959587950BC0223049F4880F991FC0
:1024200024E0813092071CF080E094E005C0803405
:10243000910514F480E490E00E947B0EA1E4B1E0E9
:10244000EDE1F1E082E101900D928150E1F710920F
:10245000730980911B0190911C01019769F41092FE
:102460001C0110921B01A3E5B1E0EDE1F1E082E176
:1024700001900D928150E1F780914B098823D9F0AA
:102480000E941930182F8823E1F080518B3058F4C6
:10249000A1E4B1E0EDE1F1E082E101900D92815023
:1024A000E1F70E946A3110924B0910927309812F53
:1024B0000E94554F06C010924A0910924D09109281
:1024C0004C09809164098770823080F40E94043244
:1024D000182F882359F010924B091092730980E449
:1024E00090E00E947B0E812F0E94554F81E0A8163C
:1024F000B104F1F48091BF04882359F08091D00495
:1025000081508093D004882321F480E090E00E94E1
:10251000A5238091D104882359F08091E204815051
:102520008093E204882321F481E090E00E94A523B7
:102530008091690990916A09019711F40E94544EA3
:1025400010926A09109269090E945C1A841995090F
:10255000409708F49DC00E945C1A2C010E94DF1A6B
:102560000E94EE1A882309F493C0179A9091620989
:10257000843141F480916309882309F089C00E9465
:10258000EB5854C0813149F49F5F80911A0189173B
:1025900008F0E4C090916309E1C0823149F4809170
:1025A0006309981719F490911A01D8C09150D6C0B8
:1025B0008331A1F480916309882339F497E09093E3
:1025C000630926E120931A01C9C0873079F587E1B4
:1025D0008093630996E290931A0122C0863189F4B0
:1025E0008091740990917509019709F051C00E947A
:1025F000AB32882311F00E94554F82E00E94EC4FCD
:1026000047C0883179F480916309873021F40E94B2
:102610003F4F97E0A3C0873109F0A0C00E944A4F06
:1026200097E19CC08F3041F40E94021A1092630916
:1026300020921A0190E092C0803151F58091640996
:102640008770823088F480917309882309F580911E
:10265000AA049091AB04A091AC04B091AD04009792
:10266000A105B105A9F002C0833091F481E0809307
:1026700073090EC0892F87500E94954C09C087317D
:1026800029F4892F87510E94064D02C00E94544EA2
:1026900080917C01882321F080917C01813099F424
:1026A00081E090E0909375098093740980916409AA
:1026B00087708250823028F41092060181E0809366
:1026C000070115981DC080917C01833029F424E016
:1026D00020937C0185E208C080917C01823031F436
:1026E00084E080937C0186E20E94554F1092750928
:1026F000109274093092060190E190930701159AA7
:102700008091970790919807892B41F080917409E7
:1027100090917509019711F4149801C0149A809151
:10272000D507882371F08091AA049091AB04A09101
:10273000AC04B091AD040097A105B10511F0139858
:1027400001C0139A0E945F15813011F416983BCC9A
:10275000169A39CC80E00E940B4C20CE90936209EF
:1027600080916309873009F08ACF84CF8EBD0DB484
:1027700007FEFDCF08952C988EBD0DB407FEFDCF4A
:102780001EBC0DB407FEFDCF8EB52C9A08952C9873
:102790008EBD0DB407FEFDCF1EBC0DB407FEFDCFF0
:1027A0008EB51EBC0DB407FEFDCF8EB52C9A0895D4
:1027B0002C98805C8EBD0DB407FEFDCF6EBD0DB4B0
:1027C00007FEFDCF2C9A08950F931F93182F0E9498
:1027D000BB13082F812F8F5F0E94BB13982F802F70
:1027E0001F910F9108950F931F93182F0E94C713E5
:1027F000082F812F8F5F0E94C713982F802F1F9162
:102800000F9108950F931F93182F072F0E94D8132D
:10281000812F8F5F602F0E94D8131F910F91089511
:102820002C9880588EBD0DB407FEFDCF6EBD0DB443
:1028300007FEFDCF2C9A08952C9880568EBD0DB4BE
:1028400007FEFDCF6EBD0DB407FEFDCF2C9A089597
:102850001F93182F8FE163E00E941C148FE1612FFA
:102860000E9410141F9108951F93182F82E00E9458
:10287000281484E1612F0E94D81382E161E00E9454
:10288000D81383E00E9428148AE00E94C71380FDB9
:10289000FBCF82E00E94281482E160E00E94D813FE
:1028A00088E10E94F3131F910895FF920F931F93E5
:1028B000F82E8B0182E00E94281484E16F2D0E9483
:1028C000D81386E1B8010E94021483E00E94281404
:1028D0008AE00E94C71380FDFBCF1F910F91FF90EC
:1028E00008952C988AE38EBD0DB407FEFDCF1EBC63
:1028F0000DB407FEFDCF8EB52C9A08952C988AE36F
:102900008EBD0DB407FEFDCF1EBC0DB407FEFDCF7E
:102910009EB51EBC0DB407FEFDCF8EB52C9A089552
:102920002C988AE38EBD0DB407FEFDCF1EBC0DB4FE
:1029300007FEFDCF9EB51EBC0DB407FEFDCF8EB5C4
:102940001EBC0DB407FEFDCF7EB51EBC0DB407FE48
:10295000FDCF6EB52C9A0895FC012C988AE38EBDAC
:102960000DB407FEFDCF20E030E008C01EBC0DB462
:1029700007FEFDCF8EB581932F5F3F4F2617370798
:10298000A8F32C9A0895982F2C988AE78EBD0DB441
:1029900007FEFDCF9EBD0DB407FEFDCF2C9A089516
:1029A000282F2C988AE78EBD0DB407FEFDCF9EBD63
:1029B0000DB407FEFDCF2EBD0DB407FEFDCF2C9A42
:1029C0000895282F2C988AE78EBD0DB407FEFDCF01
:1029D0009EBD0DB407FEFDCF2EBD0DB407FEFDCF8D
:1029E0007EBD0DB407FEFDCF6EBD0DB407FEFDCF5D
:1029F0002C9A0895FC012C988AE78EBD0DB407FE31
:102A0000FDCF20E030E008C080818EBD0DB407FE10
:102A1000FDCF2F5F3F4F319626173707A8F32C9A2B
:102A2000CB010895282F2C988AE78EBD0DB407FEA0
:102A3000FDCF80E090E005C02EBD0DB407FEFDCFB8
:102A4000019686179707C0F32C9A08958FE160E0EE
:102A50000E94D81380E160E070E00E94021482E1DD
:102A60006FEF7FE10E9402148AE06FEF7FE10E9426
:102A7000021483E00E94281487E067E00E94D813C4
:102A800087E00E94BB1380FDFBCF87E062E00E94DD
:102A90001C148FE160E30E9410148FE10E94BB13AD
:102AA00085FDFBCF80E00E94281486E10E94E4139C
:102AB00020E08750984F09F421E0822F089581E0AB
:102AC0000E94341496958795969587958170089500
:102AD0008FE10E94BB138095881F8827881F089567
:102AE000EF92FF920F931F938C0180E00E942814B5
:102AF00080E00E94F313F82EE92E60911404709187
:102B000015046A5F7F4F600F711F89E1683D780788
:102B100010F0685D794180E00E9402148F2D9E2D97
:102B20001F910F91FF90EF900895EF92FF920F93F6
:102B30001F938C0180E00E94281482E00E94F3130E
:102B4000F82EE92E0752164E82E0B8010E940214B8
:102B50008F2D9E2D1F910F91FF90EF9008950F9351
:102B60001F9300911604109117040150104080E04B
:102B70000E9428148EE160E40E941014B80189E1DB
:102B8000083D180710F067ED79E18CE00E9402140F
:102B90001F910F9108951F93CF93DF9381E00E94BF
:102BA000281489E10E94BB13182F80E00E9428148A
:102BB0008EE00E94BB13C82FD0E081E00E94281451
:102BC00089E10E94BB13181779F78CE00E94E41387
:102BD0009F718C179D0720F49C012952364E09C025
:102BE000C817D90719F427ED39E105C09C01215018
:102BF00030402C1B3D0BC901DF91CF911F910895EF
:102C0000A7E0B0E0E6E0F6E10C9497618C01E0907B
:102C10001904F0901A04E80EF91E82E0B8010E942F
:102C2000021480E00E94C31484E0B8010E940214E0
:102C300086E0B7010E9402148FE160E80E94101440
:102C40008FE160E80E941C148CE16AE00E941C1471
:102C50008FE168E00E941014809118048550823042
:102C600008F068C000E010E08CE10E94BB138A709D
:102C700031F40F5F1F4F83E0083E1807A9F78CE17E
:102C80000E94BB1381FD05C083E0083E180708F4CD
:102C900051C08FE168E00E941C1480E00E94F31391
:102CA0005C0186E00E94F3136C010894C11CD11CE6
:102CB00080E0B6010E9402148E010F5F1F4FC80111
:102CC00067E070E00E94AC14EE24F02E012F8CE13E
:102CD0000E94BB1381FF2AC08C8185FF27C08FE132
:102CE00060E80E9410148FE160E80E941C148CE1DF
:102CF0006AE00E941C148FE168E00E9410148CE1CD
:102D00000E94BB138A70D9F38FE168E00E941C1403
:102D100080E0B6010E9402148F2D902F67E070E0D2
:102D20000E94AC14E39480E1E81689F680E0B501D6
:102D30000E9402142796EAE00C94B361A0E0B0E090
:102D4000E4EAF6E10C949861B82E282F392F690136
:102D5000EE24FF24870111C00E947114D82F0E9415
:102D60007114C82FCE01A0E0B0E0E80EF91E0A1FD2
:102D70001B1F8EEF9FEFC80ED91E92E0C916D1041B
:102D800058F7C701D8019C01AD01B0FE0BC00E94ED
:102D90007114D82FC0E09E0140E050E02E0D3F1D81
:102DA000401F511F203080E0380781E0480780E055
:102DB0005807A0F0CA0140E050E0A0E0B0E0280FC2
:102DC000391F4A1F5B1F203090E0390791E0490707
:102DD00090E0590718F0C90101969C01C901CDB7CF
:102DE000DEB7E9E00C94B4610F931F938B010E944E
:102DF0007015C8010E949E169C0120953095C9014E
:102E00001F910F910895EF92FF920F931F938C01E2
:102E10007B0180E00E9428140752164E80E0B80122
:102E20000E940214C7010E949E169C0120953095B5
:102E3000C9011F910F91FF90EF900895A0E0B0E0BD
:102E4000E4E2F7E10C9499616C017B018A01411580
:102E5000510509F444C04130510551F40E947015E8
:102E6000C7010E9495150E9471140E94C31437C0B7
:102E700080E00E942814C0911404D0911504269675
:102E8000CC0DDD1D89E1C83DD80710F0C85DD941E2
:102E900080E1BE010E940214B801615070406C0FC5
:102EA0007D1F99E1683D790710F0685D794182E105
:102EB0000E94021489ED99E1E80EF91E84E1B70140
:102EC0000E9402148FE160E10E941C148FE160E215
:102ED0000E9410148FE10E94BB1385FDFBCFCDB77C
:102EE000DEB7E8E00C94B5618FE164E00E941C1449
:102EF0008DE10E94BB1382FDFBCF8FE10E94BB13CB
:102F000087FDFBCF8EE160E20E94101408951F93AD
:102F1000182F83E00E94281485E1612F0E94D813A6
:102F20001F91089583E00E94281485E10E94BB133D
:102F30000895FC012C988AE38EBD0DB407FEFDCFE9
:102F400020E030E00AC01EBC0DB407FEFDCF8EB5F8
:102F500081932F5F3F4F841719F02617370798F397
:102F600010822C9AC90108950F931F93CF93DF937A
:102F70008C01C0E0D0E003C00E9471142196C017FC
:102F8000D107D0F3DF91CF911F910F910895CF9387
:102F9000DF93EC010E94FD61AC012C988AE78EBDA5
:102FA0000DB407FEFDCF20E030E00AC0FE01E20FC5
:102FB000F31FE491EEBD0DB407FEFDCF2F5F3F4F31
:102FC0002417350798F32C9ACA01DF91CF91089501
:102FD0008EE160E20E941C1480E190E00E94551A8C
:102FE0008DE10E94BB1383FDFBCF80FFF9CF8FE102
:102FF00064E00E94101408951F938EE160E20E9425
:103000001C1480E190E00E94551A5E9880E190E0E7
:103010000E94551A5E9A80E190E00E94551A1FEFB7
:103020002C981EBD0DB407FEFDCF2C9A80E190E0D8
:103030000E94551A8DE10E94BB1383FDF1CF80FFE2
:10304000EFCF8FE160EC0E94D8138EE160E80E9420
:10305000D81388E060E070E00E9402148CE067ED15
:1030600079E10E9402148AE067ED79E10E9402147E
:1030700084E068ED79E10E94021481E00E94281446
:1030800088E161EA0E94D81382E00E94281480E05F
:103090006DE00E94D81381E060E00E94D81382E0C6
:1030A00062E30E94D8138AE06EEE75E00E9402147B
:1030B00086E062E17CE00E94021484E062E10E940A
:1030C000D81383E060E40E94D81389E06FE30E9484
:1030D000D81383E00E94281485E160E00E94D81391
:1030E00084E0609100010E94D81385E060910101A5
:1030F0000E94D81382E0609102010E94D81383E0FD
:10310000609103010E94D81380E0609104010E9445
:10311000D81381E0609105010E94D81382E10E94DA
:10312000BB138F718093180480E060E070E00E9410
:10313000551480E160E071E00E94551484E162E77B
:1031400074E00E94551480E00E9428148FE164E02E
:103150000E94D8131F910895CF93DF93EC0181E073
:103160000E94281489E10E94BB13882321F40E9445
:10317000281480E044C080E00E9428146091160466
:103180007091170480E00E940214809116049091BF
:10319000170490931504809314048EE094E066E085
:1031A00070E00E94AC1480910F048F7180930F0423
:1031B000809111048F718093110420910E0430913D
:1031C0000F043093170420931604809110049091FB
:1031D00011048F5E954080F489E1283D380760F442
:1031E00020FD0AC08091130487FD06C0809112045F
:1031F00084FD02C087FD06C00E94FC1782E0DF91BB
:10320000CF910895F89480917F0B9091800BA091BD
:10321000810BB091820B8093870790938807A093CE
:103220008907B0938A0780917D0B90917E0B9093D4
:10323000900780938F077894CE016EE070E00E9433
:10324000AC1481E0DCCF98B18F70907F892B88B966
:103250000895469898B18F70907F892B88B90000A7
:10326000449A83E090E00E94551A449808951F9371
:10327000182F88B1912F92959F70807F982B98B9C5
:10328000449A83E090E00E94551A449888B11F70D8
:10329000807F812B88B9449A83E090E00E94551A80
:1032A00044981F910895469A0E94371908954698A8
:1032B0000E94371908950E94531981E090E00E94FE
:1032C000551A0895CF93DF93EC0103C021960E9415
:1032D0005B1988818823D1F7DF91CF91089580E130
:1032E0000E94571981E090E00E94551A08958823A2
:1032F00011F48CE001C08EE00E94571981E090E04B
:103300000E94551A089581E00E94571989E190E0C2
:103310000E94551A0895662349F0613011F4805CCB
:1033200005C0623011F48C5E01C08C5A80680E9426
:10333000571981E090E00E94551A08950F931F934A
:10334000042F0E948B1910E004C080E20E945B19D8
:103350001F5F1017D4F31F910F910895682F80E01D
:1033600040E10E949E190895CF93DF93EA010E94E5
:103370008B1903C00E945B192196FE01849188235A
:10338000C9F7DF91CF9108950F931F938A010E948F
:103390008B19C8010E9462191F910F9108951F9304
:1033A000142F0E948B19812F0E94531981E090E005
:1033B0000E94551A1F9108950F931F93CF93DF9387
:1033C0008B01880F880F880F887380640E945719BB
:1033D000C0E0D0E081E090E00E94551A81E090E0EA
:1033E0000E94551AF801EC0FFD1FE4918E2F0E94E8
:1033F00053192196C830D10569F7DF91CF911F91FC
:103400000F9108951F93CF93DF9388E290E00E947D
:10341000641A83E00E94291982E490E00E94551A00
:1034200083E00E94291981E090E00E94551A83E010
:103430000E94291981E090E00E94551A82E00E94C2
:10344000291981E090E00E94551A88E20E945719DC
:1034500081E090E00E94551A88E00E94571981E0AF
:1034600090E00E94551A81E00E94571989E190E08E
:103470000E94551A86E00E94571981E090E00E9450
:10348000551A8CE00E945719C4ECD0E010E0FE0100
:1034900065917491812F0E94DC191F5F229618306C
:1034A000B1F7DF91CF911F91089528EC00002A9584
:1034B000E9F70197D1F70895F8942091BA02309175
:1034C000BB027894C9010895AC01F8942091BA0226
:1034D0003091BB02789401C0A895F8948091BA020B
:1034E0009091BB027894821B930B84179507A0F3ED
:1034F0000895DC01F8947894809187038823A9F0DB
:10350000F894E0918503F0E0EB5FFC4F80818C93B1
:10351000809185038F5F8F778093850380918703E8
:10352000815080938703789481E00895A1E0B0E012
:10353000ECE9FAE10C949D618E010F5F1F4F01C011
:10354000A895C8010E94791A8130D1F32196E4E050
:103550000C94B961A1E0B0E0E0EBFAE10C949F615A
:10356000CE0101960E94791A882311F490E022C0BE
:10357000209108042F3710F490E005C010920C043D
:1035800010920B0492E08981E22FF0E0E857FC4FA3
:103590008083E22FEF5FE09308048A3059F4F0E073
:1035A000E857FC4F10821092080410920C041092FD
:1035B0000B0491E0892F2196E2E00C94BB6190917D
:1035C000C00283B1ECEBF2E0E90FF11D80958F7042
:1035D00080839F5F93709093C00208959091BD0285
:1035E0008091BC0298238091BE0298238091BF02F3
:1035F000982341F1983011F494E11DC0943011F4F6
:1036000093E119C0923011F492E115C0913011F498
:1036100091E111C09C3011F498E10DC0933011F488
:103620009FE009C0993011F490E105C09A3011F083
:1036300090E001C096E18091920B981729F0909349
:10364000920B03C01092920B90E0892F0895EF9295
:10365000FF920F931F93CF93DF93F894E090BA02F9
:10366000F090BB0278948701A895F894C091BA02B3
:10367000D091BB027894CE01801B910B409718F03B
:103680000E94DF1A8E010E94EE1A882331F4CE19AF
:10369000DF09C051D74240F389E1CDB7DEB7E6E09C
:1036A0000C94B7610F931F93CF93DF939C01EB01B1
:1036B0008A0101C0A895F999FDCFCE01B9014FE16A
:1036C00050E00E9493621F8E8881992787FD909514
:1036D0000E94C661892B21F4CE01B8010E94F661D7
:1036E000DF91CF911F910F9108950F931F93CF9367
:1036F000DF939C01EB018A0101C0A895F999FDCFE8
:10370000CE01B9014FE050E00E9493621F8688818C
:10371000992787FD90950E94C661892B21F4CE01DF
:10372000B8010E94F661DF91CF911F910F9108952A
:10373000EF92FF920F931F93142F052FF62EE72E73
:1037400001C0A895F999FDCF0E94A3629B01AC012D
:103750002F3F8FEF38078FEF48078FEF580741F45F
:10376000212F302F4F2D5E2DC901DA019C01AD01B3
:10377000B901CA011F910F91FF90EF9008951F9317
:10378000CF93DF93EC010E94FD61182F813414F573
:103790008091030390910403019711F4A895FECF43
:1037A00081E090E0909304038093030381EC92E026
:1037B000BE010E94F6618091C1028093C600115043
:1037C0001093020381E0809301038091C100806621
:1037D0008093C100DF91CF911F9108951F93BC0189
:1037E000FC0101900020E9F731971E2F181B1134BE
:1037F0000CF58091030390910403019711F4A895AF
:10380000FECF81E090E0909304038093030381EC6A
:1038100092E00E946F628091C1028093C6001150B5
:103820001093020381E0809301038091C1008066C0
:103830008093C1001F9108951F93482F792F162F51
:10384000613444F58091030390910403019711F4CE
:10385000A895FECF81E090E090930403809303034A
:1038600021EC32E0E62FFF27E7FDF095C901642F38
:10387000AF010E942E628091C1028093C600115058
:103880001093020381E0809301038091C100806660
:103890008093C1001F9108950000000008952D9AA3
:1038A0002F98000000002F9A90E087FF02C02D9A09
:1038B00001C02D982F98000000002F9A9F5F98302C
:1038C00011F0880FF2CF08951F93CF93DF93182F35
:1038D000EB0180910D04813021F4CB010E94E43D85
:1038E000EC01F8942F9A5F9A80E30E944F1C5F9836
:1038F0002F9A5F9A1F73812F80640E944F1C80E073
:10390000D7FF02C02D9A01C02D982F98000000000B
:103910002F9A000000008F5F803119F0CC0FDD1F5F
:10392000EFCF5F982D985F9A000000001E9BFECF9E
:103930005F985F987894DF91CF911F9108951F93BE
:10394000CF93DF93C0E0D1E012E0688179812296C5
:10395000812F0E94641C1F5F1530B9F7DF91CF9152
:103960001F910895FF920F931F93182F062FF72E84
:10397000BA010E94641C812F8F5F602F7F2D0E94EF
:10398000641C1F910F91FF900895F8942F9A5F9AED
:103990008F7380680E944F1C80E020E030E02F98F9
:1039A000000000002F9A00000000220F331F1E9914
:1039B00021608F5F803199F7932F5F987894809181
:1039C0000D04813021F4822F0E94E43D9C01C90145
:1039D00008951F93CF93DF9380E00E94C51C805011
:1039E000904419F481E080930D0482E00E94C51C8C
:1039F0008F5F9F4F61F012E0C0E0D1E0812F0E9405
:103A0000C51C8883998322961F5F1530B9F7DF9113
:103A1000CF911F9108959F92AF92BF92CF92DF9264
:103A2000EF92FF920F931F93182F042FB52EA62EFF
:103A3000972E0E94C51C6C01812F8F5F0E94C51CB0
:103A40007C018FEFC8168FEFD8068FEFE8068FEF57
:103A5000F80641F4202F3B2D4A2D592DC901DA01DA
:103A60006C017D01B601C7011F910F91FF90EF908E
:103A7000DF90CF90BF90AF909F9008951F1D1F1EA5
:103A80001F1E1F1F1E1F1E1FCF93DF93EC012C96BE
:103A90004AE834D06627772736E4AEE6B1E0532F04
:103AA000537009F01197321729F078F56A0F7B1FD0
:103AB0003395F3CF4CE022D0ECE7FAE330E0C89541
:103AC0003196313011F451110A94321720F4600DFF
:103AD000711D3395F4CF402D439510D02150A8F09F
:103AE000620F711D8827992748E108D015D04CE353
:103AF00005D012D02CE302D00FD00BC03A912A91FE
:103B00002417310540F00F900F906FEF7FEF8FEF8C
:103B10009FEFDF91CF91089551E2AA1B08F4A40F03
:103B2000A79597958795779567955A95B9F7620FF9
:103B3000711D811D911D0895CF93DF93FC0120819C
:103B4000318142815381CC27DD2757FD3CC0C3E939
:103B5000DBE06CE33CD00882198239D00A821B82F8
:103B600068E135D00C821D82F9012C5F3F4F67E080
:103B70002ED00C861D869F01A6E4EEE6F1E0BA2F5A
:103B8000B37009F031972E173F0720F02E1B3F0B23
:103B9000A395F3CFAA871B862E873F87ECE7FAE32E
:103BA000AA27C8953196A13011F4B1110A942015B5
:103BB000310520F020193109A395F3CFA887198684
:103BC00023952E833F83CE01DF91CF91089500246A
:103BD00070E2220F331F441F551F001C061610F001
:103BE000061A23957A95A9F70895EBE4F4E082810B
:103BF000813041F480819181019791838083892B69
:103C000009F412823D9684E0E33BF80781F70895BA
:103C1000CF92DF92EF92FF920F931F936B017C0183
:103C20008AE290E090931A048093190480E00E9445
:103C3000281482E06DEC7FE10E9402148FEF66E0B1
:103C400070E00E94121500E011E0C80166E070E02B
:103C50000E94FA1486E098E00E94D01481E090E07F
:103C60000E94D01480E098E00E94D01486E00E9468
:103C7000C31484E00E94C31481E090E00E94D01439
:103C8000C80166E070E00E94FA146091AA04709185
:103C9000AB048091AC049091AD040E94E11480E0EB
:103CA00066E070E00E941215C701B6010E94E1149F
:103CB0008CEC9FE10E9400161F910F91FF90EF90F6
:103CC000DF90CF900895EF92FF920F931F93CF93C1
:103CD000DF937B018C01E901E1E4F4E020E08081E5
:103CE0009181A281B3818E159F05A007B10711F4C0
:103CF000922F0DC02F5F3D96283089F7CD2BF9F01C
:103D00009091A904892F8F5F87708093A9048DE01B
:103D1000989FF0011124EF5BFB4FEF012496DA012D
:103D200086E00D9009928150E1F7E082F1820283F2
:103D3000138380EB94E09387828781E08487CDB7FB
:103D4000DEB7E6E00C94B761ACE1B0E0EAEAFEE190
:103D50000C949561CE0101966CE170E00E94AC1468
:103D60008F8198850E94E43D4C016F85788989890F
:103D70009A890E94E83D5B016C01698D7A8D8B8D7B
:103D80009C8D0E94E83D7B018C0189819A810E9473
:103D9000E43D019709F071C08B819C810E94E43D54
:103DA0008050984009F069C08091AA049091AB04BA
:103DB000A091AC04B091AD04E816F9060A071B0700
:103DC00009F05BC0CE01439660E071E046E050E050
:103DD0000E947662009709F050C0AE14BF04C0067E
:103DE000D10611F482E04AC08E01075F1F4FC60161
:103DF000B501A80121E030E00E94631E81E0881631
:103E00009104D9F58CE190E090931A048093190401
:103E10008EE090E00E94951581E090E00E94D01421
:103E200080E098E00E94D01486E00E94C31484E0F1
:103E30000E94C31482E090E00E94D01480E091E0E0
:103E400066E070E00E94FA146091AA047091AB04DD
:103E50008091AC049091AD040E94E114C80166E029
:103E600070E00E94FA14CE010F9664E070E00E94A8
:103E7000FA1486E098E00E94AC1F80E06C96ECE0BB
:103E80000C94B161EF92FF920F931F93E090210485
:103E9000F090220400912304109124042091AE0498
:103EA0003091AF044091B0045091B104DA01C901DE
:103EB0008E299F29A02BB12B8F5F9F4FAF4FBF4FF4
:103EC00049F48BE194E06FEF70E046E050E00E942F
:103ED000496235C08091AA049091AB04A091AC04D2
:103EE000B091AD048E259F25A027B127822393236F
:103EF000A423B5230097A105B10511F421E009C061
:103F0000E090B204F090B3040091B4041091B504B1
:103F100022E0E1E4F4E08485813099F480819181AC
:103F2000A281B3818E159F05A007B10751F4ABE1C3
:103F3000B4E0349686E001900D928150E1F720E0E4
:103F400005C03D9684E0E93AF80729F7822F1F91D2
:103F50000F91FF90EF9008950F931F938C01809124
:103F6000190490911A040E9690931A0480931904E0
:103F700080E090E00E9495158BE194E066E070E0AF
:103F80000E94FA1480E091E066E070E00E94FA146A
:103F9000C8010E94D01488ED99E10E9400161F917B
:103FA0000F910895AEE0B0E0E8EDFFE10C949E6162
:103FB000CE0101960E94AC188823F1F0ABE1B4E089
:103FC000FE01379686E001900D928150E1F78D85D4
:103FD0009E850E94E43D28E08030920711F411E0B4
:103FE0000CC08650984031F40E94A41E182F0E94E5
:103FF000AF1503C00E94AF1510E0812F2E96E3E0AD
:104000000C94BA61A8E0B0E0E8E0F0E20C949D61A5
:1040100082E290E00E947015CE01019668E070E0A7
:104020000E94AC1489818093B9048A818093BA0478
:104030006091190470911A0482E290E00E94F416D3
:10404000892B81F08AE390E00E9470150E94901401
:104050006093BB047093BC048093BD049093BE0432
:1040600087E057C08091B904883031F16D817E813D
:104070008F8198850E94E83D9B01AC016093BB0451
:104080007093BC048093BD049093BE048091B904E6
:10409000833019F40E94FC173BC08530C9F580912C
:1040A000BA048130A9F52093B2043093B30440934D
:1040B000B4045093B5042CC04091190450911A04D3
:1040C00082E290E062E270E00E941E1782E290E0DD
:1040D0000E94951580E00E94C31480E00E94C314E2
:1040E00080E090E00E94D0146091190470911A044D
:1040F00082E290E00E9403178C0184E290E00E942B
:104100009515C8010E94D01481E00E94E72001C0EB
:104110008AE02896E4E00C94B961A0E0B0E0E3E91D
:10412000F0E20C949861B82EEB016A01E5E3F4E04B
:10413000EE24FF248701308121813296C901A0E05D
:10414000B0E0E80EF91E0A1F1B1F84E0E134F807F7
:1041500091F781E0B81651F480E00E942814C7520C
:10416000D64E80E0BE010E94021403C0CE010E9420
:104170007015C6010E949E169C0140E050E02E0D75
:104180003F1D401F511F203080E0380781E0480765
:1041900080E05807A0F0CA0140E050E0A0E0B0E0A5
:1041A000280F391F4A1F5B1F203080E0380781E04D
:1041B000480780E0580718F0C90101969C01209536
:1041C0003095C901CDB7DEB7E9E00C94B461ACE13C
:1041D000B0E0EDEEF0E20C949D61182F809119048F
:1041E00090911A04449690931A04809319048EE0D7
:1041F00090E00E94951580E095E40E94D014809193
:10420000190490911A040E94D0148091B6049091E0
:10421000B7040E94D01480E090E40E94D01480E49F
:104220000E94C314812F0E94C31480E090E00E947A
:10423000D0146091AA047091AB048091AC04909169
:10424000AD040E94E11460912104709122048091D8
:104250002304909124040E94E1148EE090E064E134
:1042600070E00E9403178C0188E190E00E94951590
:10427000C8010E94D0140E94421F882309F443C041
:10428000DE011196E9E1F4E09CE101900D9291507C
:10429000E1F7823049F46091B2047091B3048091E7
:1042A000B4049091B50408C0609121047091220477
:1042B00080912304909124040E94081E0E94AF154F
:1042C0000E945C1A8C01A8950E94D21F882311F0CD
:1042D0000E94AF150E94421F882311F420E008C0FD
:1042E0000E945C1A801B910B8858934160F326E072
:1042F000A9E1B4E0FE0131968CE101900D9281506C
:10430000E1F7222329F480E098E00E94AC1F20E02E
:104310008091B6049091B70401969093B70480936E
:10432000B604822F6C96E4E00C94B961A4E1B0E08D
:10433000ECE9F1E20C949B610E94D21F882309F4FE
:10434000A1C0823011F485E09DC08EE090E064E170
:1043500070E00E94F416892B09F091C08EE090E085
:104360000E947015CE01019664E170E00E94AC14C9
:1043700069897A898B899C890E94E83D7B018C013F
:104380002091AE043091AF044091B0045091B1043B
:104390008981682F70E0CB01807F90708034910517
:1043A00009F06DC08091AA049091AB04A091AC0477
:1043B000B091AD04E816F9060A071B0799F02E29FB
:1043C0003F29402B512B2F5F3F4F4F4F5F4F51F0F5
:1043D0008FEFE8168FEFF8068FEF08078FEF1807BB
:1043E00009F04DC06F707070660F771F660F771FF2
:1043F0006093B8048B819C810E94E43D2091B804B5
:10440000821B910990931A04809319046D857E850F
:104410008F8598890E94E83D60932104709322045F
:104420008093230490932404E0922504F0922604C0
:1044300000932704109328048091B804853120F05C
:10444000845190E00E94B41760912104709122047D
:1044500080912304909124044BE154E020E030E06B
:104460000E94631E8A85813011F482E00BC0813185
:1044700011F483E007C0863011F484E003C00E9489
:10448000AF1580E06496E6E00C94B761A0E0B0E080
:10449000ECE4F2E20C949A61D82EEB017A0184E10B
:1044A00090E0E80EF91EF0921A04E09219048CEEE6
:1044B0009FEFE80EF91E82E290E00E9495158D8133
:1044C0009E810E94D0148F8198850E94D0146985A6
:1044D0007A858B859C850E94E1146D857E858F850C
:1044E00098890E94E11480E50E94C3148D2D8F737A
:1044F0000E94C31484EB95E00E94D01460E070E049
:1045000080E090E00E94E1146091AA047091AB04F5
:104510008091AC049091AD040E94E83D6093350415
:1045200070933604809337049093380469817A81BC
:104530008B819C810E94E83D6093390470933A041A
:1045400080933B0490933C0410923D0486E080935A
:104550003E048091190490911A040E94E43D9093C6
:10456000400480933F044091190450911A0481E063
:1045700062E270E00E948D208C0182E390E00E9454
:104580009515C8010E94D01486E00E94E720682F8C
:10459000882301F58D2D90E083709070892B41F078
:1045A00089859A85AB85BC850196A11DB11D0EC07C
:1045B000E114F10479F0970140E050E089859A8593
:1045C000AB85BC85820F931FA41FB51F89879A876F
:1045D000AB87BC87862FCDB7DEB7E7E00C94B6611A
:1045E000A2E1B0E0E6EFF2E20C949F612091290491
:1045F00030912A04C901A0E0B0E08A839B83AC8398
:10460000BD8380912B0490912C049F838E833987E6
:1046100028871A861B861C861D86809131049091FE
:104620003204A0913304B09134040196A11DB11D50
:104630008E879F87A88BB98B84E0BE016F5F7F4F09
:1046400040E050E00E9446226296E2E00C94BB619A
:10465000A8E0B0E0EEE2F3E20C9495617C01809179
:104660002D0490912E040E94701500E010E06E0160
:104670000894C11CD11C2BEEA22E26E0B22EAE0C4B
:10468000BF1C92E0892E9924939453C0C60165E023
:1046900070E04AE00E949917080F191FC60169EDE2
:1046A00070E00E94ED61892B91F4E114F10419F09E
:1046B00087EE95E002C087EE94E06BEF70E04AE091
:1046C0000E949917080F191FF501908232C0C60188
:1046D00064ED70E044E050E00E940662892B19F41A
:1046E000F501808226C089818D30E1F48A818A308B
:1046F000C9F480912F049091300408171907C8F06D
:10470000EE0CFF1C87EE96E0E80EF91E81E090E0CB
:10471000F7019183808315C00F5F1F4F0E947114B2
:104720008A3039F080912F049091300408171907CE
:1047300098F380912F04909130040817190708F41A
:10474000A5CF2896ECE00C94B161CF93DF93EC01F8
:10475000009719F027EE35E002C027EE34E0FE01A5
:10476000EE0FFF1FDF0143E0AA0FBB1F4A95E1F7E1
:10477000AE0FBF1FA154BB4F1C9211961D921D92EC
:104780001D921C92149716961C921E9215971896BD
:104790001C921E9217971D961D921D921D921C929F
:1047A000509780E091E0D901AC011D9241505040FA
:1047B000E1F7E951F94F11821082C551D94F1882A2
:1047C000DF91CF910895A6E2B0E0E9EEF3E20C9418
:1047D00091610091B80410E0025F1F4FCE01439633
:1047E00064E170E00E94AC148B899C890E94E43DD6
:1047F00090932A04809329048D899E890E94E43D28
:1048000090932C0480932B046F89788D898D9A8DD9
:104810000E94E83D60933104709332048093330426
:10482000909334042F8D2695269530E0C801820F91
:10483000931F90932E0480932D04809119049091DE
:104840001A04821B930B9093300480932F04609181
:1048500021047091220480912304909124040E94E9
:10486000E83D609335047093360480933704909349
:10487000380460912504709126048091270490915A
:1048800028040E94E83D6093390470933A048093B1
:104890003B0490933C0410923D0486E080933E04D8
:1048A0008091190490911A040E94E43D9093400471
:1048B00080933F044091190450911A0480E0B8019C
:1048C0000E948D20892B09F099C198A1992309F4A0
:1048D00095C16090210470902204809023049090F0
:1048E0002404E0902904F0902A04A0902B04B090B6
:1048F0002C040FEB14E0CC24DD246FEF7FEF2E01AE
:104900000894411C511CD201F80182E101900D92E2
:104910008150E1F7AE81BF81E885F9852A813B812D
:104920004C815D818981882331F48FEF6F3F780757
:1049300011F4B6010BC0261537054805590531F4A9
:10494000EE15FF0519F4AA15BB05C1F00894C11CAA
:10495000D11C0E5E1F4FE2E0CE16D104A1F6FFEF90
:104960006F3F7F0741F06B01C094D0948CE9C8166B
:104970008FEFD80619F40E94F022FFC0D7FE47C07F
:1049800091FF3FC18091E3049091E404A816B90619
:1049900009F037C1C094D094C601880F991F8C01CB
:1049A00043E0000F111F4A95E1F7080F191F01544A
:1049B0001B4FF8016182728283829482B682A58243
:1049C000F086E78281E080830E94733DF801618771
:1049D0007287838794878091310490913204A091EB
:1049E0003304B09134040196A11DB11D85879687CB
:1049F000A787B08B8CE3818B82E1B80140E050E067
:104A00000E944622F82E882309F4FCC053C091FF6F
:104A100003C00E94F0224DC092FF0FC0B601660F86
:104A2000771FCB0123E0880F991F2A95E1F7680FC4
:104A3000791F61547B4F84E038C090FF3FC0C601AE
:104A4000880F991F8C01B3E0000F111FBA95E1F791
:104A5000080F191F01541B4FF80120818091310468
:104A600090913204A0913304B09134040196A11DB9
:104A7000B11D85879687A787B08B223079F480E1B6
:104A8000B80140E050E00E94462281E1B80140E0D8
:104A900050E00E944622F82E85E0A1C0233019F094
:104AA000263009F0AEC080E1B80140E050E00E943D
:104AB0004622F82EC6010E94A523A4C093FF5FC022
:104AC00080912F0490913004009711F480E055C03C
:104AD0005601AA0CBB1C8501F3E0000F111FFA95CB
:104AE000E1F70A0D1B1D01541B4FF80120812130F5
:104AF00019F482E0808302C0223011F0FF243CC010
:104B0000A0E0B0E0209131043091320440913304B0
:104B100050913404820F931FA41FB51FF80185879D
:104B20009687A787B08B258136818091E304909189
:104B3000E40428173907B1F480E1B80140E050E0FF
:104B40000E944622F82EC6010E942823F501E95151
:104B5000F94F80819181019779F4C6010E94CF4479
:104B6000F82E0AC081E1B80140E050E00E944622E0
:104B7000F82E83E0F80180838F2DF82E43C094FF38
:104B800040C0C601880F991F8C0173E0000F111FF0
:104B90007A95E1F7080F191F01541B4FF801808126
:104BA000813011F482E022C08230E1F480912F0440
:104BB00090913004892B59F080E1B80140E050E039
:104BC0000E944622F82EC6010E9428231BC081E1C4
:104BD000B80140E050E00E944622F82E83E0F80140
:104BE000808310C0833021F486E0F801808309C0FF
:104BF000853039F4C6010E94A52303C068E0F62E73
:104C000001C0FF248F2DA696E0E10C94AD61CF93F7
:104C1000DF93089690931A048093190482E290E03F
:104C20000E94951580912B0490912C040E94D01421
:104C30008091290490912A040E94D0148091190433
:104C400090911A040E94D01480E090E00E94D01449
:104C50006091AA047091AB048091AC049091AD0472
:104C60000E94E83D609335047093360480933704C6
:104C70009093380460912104709122048091230460
:104C8000909124040E94E83D6093390470933A04A3
:104C900080933B0490933C0410923D0481E1809307
:104CA0003E048091190490911A040E94E43D90936F
:104CB000400480933F044091190450911A0481E00C
:104CC00062E270E00E948D20EC01009711F4CFEFBA
:104CD000DFEF88E290E00E949515CE010E94D0148B
:104CE00081E10E94E720DF91CF910895A0E1B0E03B
:104CF000ECE7F6E20C949B61CE01099668E070E067
:104D00000E94AC1489859A850E94E43D90932A0400
:104D1000809329048B859C850E94E43D90932C040C
:104D200080932B048D859E850E94E43D8C01085064
:104D300010401093300400932F04085F1F4F8091A0
:104D4000B804E82EFF248EE090E0E80EF91E8F856F
:104D50009889892BB9F16091210470912204809186
:104D60002304909124040E94E83D609335047093DD
:104D70003604809337049093380460912504709131
:104D8000260480912704909128040E94E83D6093B6
:104D9000390470933A0480933B0490933C0410923E
:104DA0003D0481E180933E048D859E85909340046F
:104DB00080933F0480E0B701A8010E948D20892BD9
:104DC00009F04AC0C701089690932E0480932D04E1
:104DD00020912B0430912C042B37310519F40E94BB
:104DE00063333DC02532310519F40E94333B37C08F
:104DF00044E02030340719F40E94D52C30C024340C
:104E0000310519F40E94952A2AC02938310519F470
:104E10000E941D2E24C02151374201F50E947015B9
:104E20008E010F5F1F4FC80167E070E00E94AC1455
:104E3000C80168EE70E047E050E00E940662892BEE
:104E400069F48AE290E00E9495158FED90E00E944F
:104E5000C7170E940726FFCF89E001C080E0609657
:104E6000E6E00C94B7618091AA079091AB07A091FE
:104E7000AC07B091AD078093210490932204A093D6
:104E80002304B093240483E490E090932A04809355
:104E9000290484E490E090932C0480932B048AE20C
:104EA00090E00E94951560E076E081E091E00E943C
:104EB000E1140E94733D6093BE077093BF07809317
:104EC000C0079093C1070E94E11480E090E00E9427
:104ED000D01480E090E00E94D01460E070E080E0A8
:104EE00090E00E94E11480E06CE070E00E941215F6
:104EF00080E091E066E070E00E94FA1480E06AECE5
:104F000070E00E94121563E673E582E893E60E9462
:104F1000E11481E095E30E94D01484E00E94C31460
:104F200082E30E94C31484E00E94C3146091AA0427
:104F30007091AB048091AC049091AD040E94E11497
:104F400086E30E94C31484E00E94C3146091AA0700
:104F50007091AB078091AC079091AD070E94E1146E
:104F60008FEF0E94C31480E06CE270E00E94121583
:104F70008CE291E00E94072608950F931F9381E031
:104F80008093D5078FEF9FEFAFEFBFEF80932104A2
:104F900090932204A0932304B093240483E490E02C
:104FA00090932A048093290484E490E090932C0445
:104FB00080932B041092AE041092AF041092B004B0
:104FC0001092B1041092AA041092AB041092AC0497
:104FD0001092AD0410925E0910925F091092600960
:104FE000109261091092B2041092B3041092B404AA
:104FF0001092B5041092A6071092A7071092A80766
:105000001092A9071092A2071092A3071092A4076A
:105010001092A5071092AE071092AF071092B0073A
:105020001092B1071092AA071092AB071092AC072A
:105030001092AD071092BA071092BB071092BC07EE
:105040001092BD071092B2071092B3071092B407E6
:105050001092B5071092B6071092B7071092B807D2
:105060001092B9071092CA071092CB071092CC0782
:105070001092CD071092D8070E94733D6093BE072F
:105080007093BF078093C0079093C1078AE290E0B6
:105090000E94951560E076E081E091E00E94E114C5
:1050A0006091BE077091BF078091C0079091C107C2
:1050B0000E94E11460E070E880E090E00E94E1145A
:1050C00080E060E170E00E94121500E011E0C8018C
:1050D00066E070E00E94FA1480E06AEC70E00E94E2
:1050E000121563E673E582E893E60E94E11481E01D
:1050F00095E30E94D01481E00E94C3148DE30E94C6
:10510000C31487E00E94C31481E00E94C314C80145
:1051100066E070E00E94FA148FEF0E94C31480E0F2
:105120006FE270E00E9412158CE291E00E94072667
:105130001F910F9108950F931F93182F8093D507F8
:10514000883129F08FEF9FEFAFEFBFEF08C080915C
:10515000AA079091AB07A091AC07B091AD078093DF
:10516000210490932204A0932304B09324041330C9
:1051700051F00E94733D6093BE077093BF07809308
:10518000C0079093C107EEE4F9E001900020E9F731
:105190003197EE54F9400E2F0F5F83E490E0909327
:1051A0002A048093290484E490E090932C04809353
:1051B0002B048AE290E00E94951560E076E081E0A1
:1051C00091E00E94E1146091BE077091BF07809149
:1051D000C0079091C1070E94E11480E090E00E9416
:1051E000D014183119F080E090E802C080E090E01F
:1051F0000E94D0146091AA047091AB048091AC0419
:105200009091AD040E94E11480E06CE070E00E9497
:10521000121580E091E066E070E00E94FA1480E0F0
:105220006AEC70E00E94121563E673E582E893E68B
:105230000E94E11481E095E30E94D01483E00E9473
:10524000C3148CE00E94C314802F0E94C3148EE408
:1052500099E0602F70E00E94FA14133019F582E390
:105260000E94C31484E00E94C31480912D04909185
:105270002E0440960E9470150E9490140E94E11422
:1052800086E30E94C31484E00E94C3146091AA07BD
:105290007091AB078091AC079091AD070E94E1142B
:1052A00019E115C0163111F015E211C082E30E9418
:1052B000C31484E00E94C31460919E0770919F07FD
:1052C0008091A0079091A1070E94E1141FE187E35C
:1052D0000E94C31486E00E94C31481E00E94C3149C
:1052E00083E00E94C31486E00E94C31483E30E94FB
:1052F000C3148AE30E94C3148BE30E94C3148DE39A
:105300000E94C31487E00E94C31481E00E94C3146A
:1053100080E091E066E070E00E94FA148FEF0E9456
:10532000C314101B80E0612F70E00E9412158CE204
:1053300091E00E9407261F910F910895EF92FF922E
:105340000F931F938091D6079091D707892B59F41B
:10535000A8E0B1E0EDE1F1E082E101900D92815031
:10536000E1F760E0DCC08091D507813031F0863113
:1053700021F0883111F08931D9F5E090D207F09011
:10538000D30700E010E088E091E06DE171E00E9459
:10539000813EE61AF70A080B190BE092CE07F0924D
:1053A000CF070093D0071093D1071E141F041006D7
:1053B0001106F4F08091D507813049F0863159F417
:1053C0008091D8078F5F8093D807833018F00E94B0
:1053D000BD2703C086E10E949B28682FA8E0B1E0AA
:1053E000EDE1F1E082E101900D928150E1F701C021
:1053F00060E0E090CA07F090CB070091CC071091D5
:10540000CD07D801C7010196A11DB11D0297A105C5
:10541000B10508F484C08091C2079091C307A091A0
:10542000C407B091C5072091C6073091C7074091C6
:10543000C8075091C9070097A105B10591F10197DF
:10544000A109B1098093C2079093C307A093C40731
:10545000B093C50721503040404050402093C607CC
:105460003093C7074093C8075093C9070894E108D1
:10547000F10801091109E092CA07F092CB070093E5
:10548000CC071093CD070097A105B10509F047C0DF
:1054900088E10E949B28682F882309F040C06CE0B7
:1054A0003EC00894E108F1080109110921153105F0
:1054B0004105510509F1DA01C9010197A109B109B5
:1054C0008093C6079093C707A093C807B093C907F6
:1054D000E092CA07F092CB070093CC071093CD0758
:1054E0000097A105B105D9F489E10E949B28682F96
:1054F0008823A9F46DE013C0E092CA07F092CB07AD
:105500000093CC071093CD07E114F10401051105B8
:1055100031F40E94BD27682F882309F46EE0862F9E
:105520001F910F91FF90EF900895ACE1B0E0EBE98F
:10553000FAE20C949B618091D507882309F4E8C1B5
:10554000873109F4E5C180912D0490912E0480519A
:105550009F4F0E9470150E947114182F8F3F09F4FD
:10556000C5C00E947114082F153341F4813009F031
:10557000D6C10E9471148093D407EDCF113071F41D
:10558000843009F0CCC10E9490146093A2077093FC
:10559000A3078093A4079093A507DDCF133071F480
:1055A000843008F4BCC10E9490146093A6077093E5
:1055B000A7078093A8079093A9071FC0163371F41B
:1055C000843008F4ACC10E9490146093AA077093D1
:1055D000AB078093AC079093AD070FC01630A1F4D2
:1055E000843008F49CC10E9490146093AE077093BD
:1055F000AF078093B0079093B107043009F4ABCFA5
:10560000802F90E004976FC0133309F04BC08430B3
:1056100009F0A1CF0E9490147B018C016093BA071E
:105620007093BB078093BC079093BD078091B6072A
:105630009091B707A091B807B091B9070097A1055D
:10564000B105B1F4C801B7012BE633E040E050E00A
:105650000E94136128EE33E040E050E00E94526166
:105660002093B6073093B7074093B8075093B90714
:105670008091B2079091B307A091B407B091B5079C
:105680000097A105B10509F066CF16950795F79427
:10569000E794E092B207F092B3070093B407109337
:1056A000B50759CF1A3371F4843009F054CF0E94F2
:1056B00090146093B2077093B3078093B4079093EC
:1056C000B50749CF1B3371F4843009F044CF0E94F1
:1056D00090146093B6077093B7078093B8079093C0
:1056E000B90739CF90E00E94B41735CF80912D04CF
:1056F00090912E0404960E9470158091D507909188
:10570000D4078130B9F4923009F004C10E9490149A
:105710002091BE073091BF074091C0075091C1074B
:10572000621773078407950709F0F4C083E00E94AD
:105730009B28F1C0953009F0D9C00E9490142091A7
:10574000BE073091BF074091C0075091C107621753
:1057500073078407950709F0DDC087E18093D507BB
:1057600080912D0490912E0440960E9470150E9405
:105770009014AB01BC014093AA045093AB04609316
:10578000AC047093AD0488E090E00E94D1628091F7
:10579000A2079091A307A091A407B091A5078093B9
:1057A000AE049093AF04A093B004B093B104809181
:1057B000A6079091A707A091A807B091A907809389
:1057C000B2049093B304A093B404B093B504809151
:1057D000AE079091AF07A091B007B091B107809349
:1057E0005E0990935F09A0936009B093610980916D
:1057F000B2079091B307A091B407B091B507809319
:10580000C2079093C307A093C407B093C5078091C4
:10581000B6079091B707A091B807B091B9078093E8
:10582000C6079093C707A093C807B093C907809194
:10583000BA079091BB07A091BC07B091BD078093B8
:10584000CA079093CB07A093CC07B093CD078F5F87
:105850009F4FAF4FBF4F21F41092D7071092D6073A
:10586000DE011196E9E1F4E08CE101900D928150A6
:10587000E1F76091AA047091AB048091AC0490911F
:10588000AD040E94081E0E94AF150E945C1A8C0194
:10589000A8950E94D21F813019F40E94AF1509C04B
:1058A000823039F40E9433278823B1F40E94BD2747
:1058B00013C00E945C1A801B910B8D54914040F3E1
:1058C000809162098150823030F481E090E09093C1
:1058D0006A098093690980E0A9E1B4E0FE0131968C
:1058E0009CE101900D929150E1F715C0963091F432
:1058F0000E9490142091BE073091BF074091C007CD
:105900005091C107621773078407950719F407C000
:1059100080E001C08FE06C96E6E00C94B7610E94D5
:10592000BD27F9CFAF92BF92DF92EF92FF920F9314
:105930001F93DF93CF930F92CDB7DEB7F82EE92EEA
:105940009C0159018EE2D82E0E947114982F882351
:1059500031F40894A108B108F501108219C0807CC7
:10596000803C11F085010AC00E94711411C0998316
:105970000E947114F80181938F019981802F8A19F7
:105980008917A8F3A90EB11CF501D1925F01DCCFF4
:105990008F2D9E2D0F90CF91DF911F910F91FF9032
:1059A000EF90DF90BF90AF900895ACE4B0E0EBEDE6
:1059B000FCE20C94916180912D0490912E040E9440
:1059C0007015CE0101966CE070E00E94AC148981E4
:1059D0009A810E94E43D2091430930914409821745
:1059E000930709F06AC08D819E810E94E43D6C019D
:1059F000EE24FF243DE2A32EB12CAC0EBD1E2DE003
:105A0000822E912C8C0E9D1E14C0C5010E94922CDA
:105A10000E947E148C010E947E140130110531F425
:105A2000019721F4C401B5010E946F620894E11C42
:105A3000F11CEC14FD0448F38F8198850E94E43D2D
:105A40003C01EE24FF249DE2492E512C4C0E5D1E9C
:105A500031C0C2010E94922C0E947E148C010E94CF
:105A60007E144C010E9490145B016C010E947E1414
:105A700001301105D1F421E082169104B1F4843093
:105A8000910599F40E949014AB01BC014093450923
:105A9000509346096093470970934809CE010D96CB
:105AA000960185010E94FB3008C00E94B41708943B
:105AB000E11CF11CE614F70460F280E0C45BDF4FE8
:105AC000E0E10C94AD61AF92BF92DF92EF92FF9252
:105AD0000F931F93CF93DF93182F092F80915E09A7
:105AE00090915F09A0916009B091610980932104B0
:105AF00090932204A0932304B093240485E390E0C0
:105B000090932A048093290480E094E090932C04DD
:105B100080932B040E94733D709344096093430962
:105B20008AE290E00E949515809143099091440982
:105B30000E94D01480E091E00E94D01481E090E0B7
:105B40000E94D01480E090E00E94D01480E090E0A9
:105B50000E94D01480E090E00E94D014212F302FBA
:105B6000C901EC0140E1A42EB12C7E010E2D0C1BCD
:105B7000F701D080FEE2DF1631F0DD2021F008943D
:105B8000E11CF11CF3CF802F0E94C31410E0CE0162
:105B9000B8010E94FA140F5F1F4FA00EB11EDD2046
:105BA00019F0E7012196E1CF80E00E94C31481E063
:105BB00090E00E94D01481E090E00E94D014C501D2
:105BC00001960E940726DF91CF911F910F91FF90C0
:105BD000EF90DF90BF90AF9008951F930E947114D3
:105BE000182F11541295107F0E94711481548F70D8
:105BF000812B1F9108950F931F93CF93DF93EC0197
:105C000000E0899190E00E94DA61182F85958595D2
:105C1000859585958F5B0E94C3141F70812F8F5BC4
:105C20000E94C3140F5F003161F780E00E94C3142B
:105C3000DF91CF911F910F910895ACE1B0E0E3E2C5
:105C4000FEE20C94916180912D0490912E040E94AB
:105C50007015CE0101966CE070E00E94AC148B814F
:105C60009C810E94E43D9C018F709070892B11F003
:105C700082E1EEC037FF5AC089819A810E94E43DDB
:105C800020914309309144098217930709F0DFC03E
:105C90008F8198850E94E43D019711F080E1D8C082
:105CA0000E947114803211F081E1D2C08E01035F35
:105CB0001F4FC801902E892E2DE1E22EF12CEC0E03
:105CC000FD1E0E94ED2DF80181938F01EE15FF0559
:105CD000C1F71C8E0E9471140E947E148C010E94D8
:105CE0007E147C010E9490145B016C01003211054E
:105CF00009F0ADC0F1E0EF16F10409F0A8C00E9470
:105D00007E140E947E140E949014AB01BC0140934B
:105D10004509509346096093470970934809892DB6
:105D2000982D960185010E94FB3091C02070387734
:105D3000232B09F08CC080912F0490913004C297DE
:105D400009F085C089819A810E94E43D4C018D81D2
:105D50009E810E94E43D5C01CC24DD249DE0692EFF
:105D6000712C6C0E7D1E8DE1482E512C4C0E5D1E4B
:105D700031C00E947114803209F069C083010E9411
:105D8000ED2DF80181938F01E415F505C1F71C8E07
:105D90000E9471140E947E147C010E947E1401975F
:105DA000B1F4F0E2EF16F10451F4C3016EE479E0CE
:105DB0000E946662009759F400E015E84FC081E246
:105DC000E816F10421F48D858A3209F445C008945F
:105DD000C11CD11CCA14DB0460F239C086E090E01B
:105DE0000E94D01480E090E00E94D0146091AA0438
:105DF0007091AB048091AC049091AD040E94E114C9
:105E00008EE390E021C08DE390E00E94D01481E009
:105E10000E94C3148EE499E06FE070E00E94FA14CF
:105E200080E00E94C31480E094E00E94D01480E0DF
:105E300091E066E070E00E94FA1480E064E270E0B5
:105E40000E94121585E790E00E94072601C080E0BD
:105E50006C96E0E10C94AD6100E014E88AE290E019
:105E60000E949515C4010E94D014C8010E94D0144C
:105E700080E090E00E94D01481E090E00E94D01475
:105E800080E090E00E94D01480E090E00E94D01466
:105E900080E20E94C314CE010D960E94FB2DC70123
:105EA0000E94D01481E090E00E94D01468E572E076
:105EB00080E090E00E94E114E0E2EE16F10409F0C7
:105EC000A2CF8CCF0F931F938C018091AE04909141
:105ED000AF04A091B004B091B10480959095A095C5
:105EE000B0952091AA043091AB044091AC0450913C
:105EF000AD04822B932BA42BB52B8093210490937C
:105F00002204A0932304B093240489E890E09093A2
:105F10002A048093290490932C0480932B040E94DC
:105F2000733D70934409609343098AE290E00E94B4
:105F3000951580914309909144090E94D01480E105
:105F400091E00E94D01481E090E00E94D01480E0A3
:105F500090E00E94D01480E090E00E94D01480E095
:105F600090E00E94D01480E20E94C314C8010E94F5
:105F7000FB2D80E290E00E94D01481E090E00E942E
:105F8000D01482E390E00E9407261F910F9108959C
:105F9000EDE1F8E084818130A1F480819181A281DA
:105FA000B3810097A105B10561F00197A109B1097D
:105FB00080839183A283B3830097A105B10509F47F
:105FC0001482B99689E0E536F80721F70895A9E229
:105FD000B0E0EDEEFFE20C9499617C0109EF17E06F
:105FE0006E010894C11CD11CD601F80189E2019010
:105FF0000D928150E1F789A5813059F4C601B701AE
:106000000E946662009729F429A13AA14BA15CA1E4
:106010000AC0075D1F4F89E00134180729F720E007
:1060200030E040E050E0B901CA01A996E8E00C94E4
:10603000B561CF93DF9380914B09813001F5C9EDB4
:10604000D7E0CE0165E479E00E94EE3D813009F4AD
:10605000C3C0FE0101900020E9F73197EC1BFD0B56
:10606000709738F4CE016EE270E00E945B62009798
:1060700011F084E001C082E080934B09A9C0823016
:1060800009F589ED97E00E94E72F60934509709329
:106090004609809347099093480961157105810568
:1060A000910509F099C00E945C1A9093420980936F
:1060B000410989ED97E00E94622F282F10924A092A
:1060C00083E053C0833079F580914509909146096A
:1060D000A0914709B09148090097A105B10509F0C1
:1060E0007BC00E945C1A2091410930914209821BB9
:1060F000930B885E934008F46BC080914A098F5FD0
:1061000080934A09833020F0209171072D5E61C091
:106110000E945C1A909342098093410989ED97E0AF
:106120000E94622F53C0843019F589ED97E00E94D8
:10613000E72F609345097093460980934709909330
:106140004809611571058105910509F045C00E9456
:106150005C1A909342098093410989ED97E00E946F
:10616000632D282F10924A0985E080934B0931C096
:10617000853071F58091450990914609A0914709B4
:10618000B09148090097A105B10531F50E945C1A4C
:106190002091410930914209821B930B885E934004
:1061A000B8F080914A098F5F80934A09833020F0CC
:1061B00020917107295E0DC00E945C1A90934209DC
:1061C0008093410989ED97E00E94632D282F01C03B
:1061D00020E080E090E003C020E081E090E0909338
:1061E0004D0980934C09019711F410924B09822FAD
:1061F000DF91CF910895A0E0B0E0E1E0F1E30C94ED
:106200009361EC016A017B014801590100E010E053
:1062100089E2682E712C069DC001079D900D169D88
:10622000900D11248750984FBE010E94666200971E
:1062300039F10F5F1F4F0830110569F720914909A7
:10624000822F8F5F87708093490930E089E290E068
:10625000289F8001299F100D389F100D1124075091
:10626000184FC801BE010E946F62F801C0A2D1A2FE
:10627000E2A2F3A284A295A2A6A2B7A281E080A77F
:10628000CDB7DEB7EEE00C94AF61A8E0B0E0EBE490
:10629000F1E30C9497616D837E838F8398871982D5
:1062A0001A821B821C8229813A814B815C81F8EE23
:1062B000AF2EE3E0BE2ECC24DD24EE24FF2400E04C
:1062C00010E00E949E5A952FB901842F2896EAE08B
:1062D0000C94B361A4E2B0E0E0E7F1E30C949961BF
:1062E000109171071093720700E0B5E0EB2EF12CCE
:1062F000EC0EFD1E6E010894C11CD11C1F5F1370B3
:10630000E12FF0E0EE0FFF1FEC5AFE4F6591749104
:10631000C7010E946F62C701B6010E94EE3D813045
:1063200041F489819A81AB81BC810097A105B105B7
:1063300019F01093710703C00F5F0430F9F6A496AB
:10634000E8E00C94B561AF92BF92CF92DF92EF92EA
:10635000FF920F931F936093210470932204809304
:106360002304909324048BE790E090932A04809375
:10637000290490932C0480932B048AE290E00E94DD
:10638000951583E20E94C31480E067E270E00E94EA
:106390001215F894E0907F0BF090800B0091810B28
:1063A0001091820B60917D0B70917E0B882777FD99
:1063B0008095982F0E9445315B016C017894609321
:1063C000830770938407809385079093860780E8FE
:1063D0009EE7AAEAB3E8E80EF91E0A1F1B1FC801D0
:1063E000B7010E94E114C601B5010E94E11480E3E7
:1063F00090E00E9407261F910F91FF90EF90DF9091
:10640000CF90BF90AF9008951F93109173091123FF
:1064100009F480C01130A1F480917107E82FF0E0F9
:10642000EE0FFF1FEC5AFE4F6591749189ED97E0D6
:106430000E946F6210934B0982E0809373096AC0D7
:10644000123089F580914C0990914D09019709F01E
:1064500061C010924D0910924C09609145097091EC
:10646000460980914709909148096093ED06709321
:10647000EE068093EF069093F00610929B070E9421
:10648000A331182F882351F483E0809373090E946D
:106490005C1A909394078093930702C0109273093B
:1064A0000E946A3138C01330A9F50E945C1A20910D
:1064B000930730919407821B930B2091950730919D
:1064C00096078217930730F180919B078F5F809327
:1064D0009B07833040F010937D0110917207145E8A
:1064E0000E946F0B18C06091ED067091EE068091CE
:1064F000EF069091F0060E94A331182F882339F4FB
:106500000E945C1A909394078093930704C01092A2
:10651000730901C010E0812F1F91089580916409D3
:106520008770823019F484EF90E004C0833041F426
:1065300080EF90E00E94C71780E00E94C314089586
:106540006091AA047091AB048091AC049091AD0469
:106550000E94E1140895AF92BF92CF92DF92EF9222
:10656000FF920F931F938091770790917807A091E6
:106570007907B0917A078093210490932204A09325
:106580002304B09324048BE790E090932A04809333
:10659000290490932C0480932B048091740990918A
:1065A0007509892B19F405EE10E102C005E211E02E
:1065B0008AE290E00E949515802F0E94C314812FDB
:1065C0000E94C314609197077091980720E030E80B
:1065D0004FE0C90186239723892B29F4415019F0F4
:1065E00036952795F6CF842F0E94C31486EF0E941C
:1065F000C31460917B0770917C0780917D07909117
:106600007E070E94E11460917F077091800780915E
:106610008107909182070E94E1140E948E3260915E
:1066200091077091920780E090E00E9445317B01D4
:106630008C0160918B0770918C0780918D079091F0
:106640008E076058714885459C470E94E114C80137
:10665000B7010E94E11480E060E170E00E94121531
:10666000F894E0907F0BF090800B0091810B1091DB
:10667000820B60917D0B70917E0B882777FD809552
:10668000982F0E9445315B016C01789480E89EE769
:10669000AAEAB3E8E80EF91E0A1F1B1FC801B701DA
:1066A0000E94E114C601B5010E94E11480E390E06C
:1066B0000E9407261F910F91FF90EF90DF90CF90DF
:1066C000BF90AF900895ABE6B0E0E9E6F3E30C9439
:1066D0008F6180912D0490912E040E947015CE013F
:1066E000819660E370E00E94AC1499A1892F8770B5
:1066F000843009F01CC480917309882309F4ADC764
:10670000892F807C809306019AA1803C21F09923F7
:1067100011F0903158F082E080937D0110924B0986
:10672000109273090E946F0B8BE198C79F5F909343
:1067300007016DA17EA18FA198A50E94E83D6093FD
:106740007B0770937C0780937D0790937E0769A5F4
:106750007AA58BA59CA50E94E83D60937F07709366
:1067600080078093810790938207FE01E05CFF4FD2
:1067700090812FAD5EAD6DAD7CADABADDAAC99ACBB
:10678000FE01EC5BFF4FC080FE01ED5BFF4FB08070
:10679000FE01EE5BFF4FA080FE01EF5BFF4F7080BC
:1067A000FE01E85BFF4F8081FE01E95BFF4F308116
:1067B000FE01EA5BFF4F4081FE01EB5BFF4FE08192
:1067C000E82EE91A91E08E1508F090E0832F821BE5
:1067D00021E0381708F020E0F82EF91A91E08F1523
:1067E00008F090E0292B842F851B31E0481708F032
:1067F00030E0082F021B91E0801708F090E0392B61
:106800008E2F861B21E0E81708F020E0182F131BBD
:1068100091E0811708F090E0292B8C2D871B31E047
:10682000C81608F030E0B82FB21B91E08B1708F0C3
:1068300090E0392B8B2D8A1B21E0B81608F020E060
:10684000A82FA31B91E08A1708F090E0292B8A2D2E
:106850008D1991E0A81608F090E0F82FF21B21E0C6
:106860008F1708F020E0922BE72DE919E91B97011B
:10687000A8016B2F7A2F8F2F9E2F52F52E2D2F5F71
:1068800081E02E1508F080E0382F3F0D81E03F15A4
:1068900008F080E0482F400F81E0401708F080E0CA
:1068A000582F510F81E0511708F080E0682F6B0FCF
:1068B00081E06B1708F080E0782F7A0F81E07A177B
:1068C00008F080E08F0F91E08F1708F090E09E0FA6
:1068D00001E00E94195A622E532E442E352E262E88
:1068E00066967FAF669767968FAF679768969FAFFC
:1068F0006897FE01E45BFF4FC080FE01E55BFF4F40
:10690000B080FE01E65BFF4FA080FE01E75BFF4F1A
:106910007080FE01E05BFF4F0081FE01E15BFF4FF5
:10692000F080FE01E25BFF4F9080FE01E35BFF4FD2
:1069300080808091870790918807A0918907B09106
:106940008A0780589148A545BC47182F8D8B9E8B90
:10695000AF8BB88F60918F077091900780E090E0C7
:106960000E944531698B7A8B8B8B9C8B872F3B895F
:10697000492F5E897F89E88DD02ED61A91E00D15BA
:1069800008F090E02F2D281B822F21E0F81608F048
:1069900020E0E82EE91A91E08E1508F090E0292B0E
:1069A000892D831B31E0981608F030E0F82EF21A9A
:1069B00091E08F1508F090E0392B882D841B21E0A1
:1069C000881608F020E0082F031B91E0801708F0DC
:1069D00090E0292B3C2D311B132F91E0C31608F0BA
:1069E00090E0B12FB21B81E01B1708F080E0982BDC
:1069F0008B2D851B21E0B81608F020E0A82FA91BDD
:106A000091E08A1708F090E0292B8A2D871B91E0EE
:106A1000A81608F090E0F82FF21B21E08F1708F07D
:106A200020E0922B7E1AE72DE91B2D2D3E2D4F2DB8
:106A3000502F6B2F7A2F8F2F9E2F52F52D2D2F5FDA
:106A400081E02D1508F080E0382F3E0D81E03E15E5
:106A500008F080E0482F4F0D81E04F1508F080E0EE
:106A6000582F500F81E0501708F080E0682F6B0F0F
:106A700081E06B1708F080E0782F7A0F81E07A17B9
:106A800008F080E08F0F91E08F1708F090E09E0FE4
:106A900001E00E94195AA32FB42F152F062FF72EAD
:106AA000D82EC22EC60CF1E0C21608F0F0E03A2F44
:106AB000350DE1E03A1708F0E0E0EF2EE30E21E0BB
:106AC000E31608F020E0E22B4B2F440D31E04B178A
:106AD00008F030E0AE2FA40F21E0A41708F020E06A
:106AE000322B512F530D41E0511708F040E0F32FA6
:106AF000F50F21E0F51708F020E0422B602F620D22
:106B000031E0601708F030E0E42FE60F21E0E617EF
:106B100008F020E0322B66967FAD66977F0D41E04E
:106B20007F1508F040E0532F570F21E0571708F06A
:106B300020E0422B67968FAD67978D0D21E08D1574
:106B400008F020E0480F31E0481708F030E0232B30
:106B500068968FAD6897980F290FC98AEA8AAB8B20
:106B6000FC8BED8B5E8B4F8B288F4D885E886F88FA
:106B7000788C89899A89AB89BC894C015D01CC24C8
:106B8000DD2476019C01A50160E070E080E090E0EA
:106B900002E00E949A59122F232E69964FAF6997EF
:106BA0006A965FAF6A976B966FAF6B976C967FAF85
:106BB0006C976D968FAF6D976E969FAF6E9705E051
:106BC0000E949A59A32FB42F052F6F966FAF6F971E
:106BD000A0967FAFA097A1968FAFA197A2969FAFE7
:106BE000A297322E311AF1E0231508F0F0E03A2F87
:106BF0003219E1E0A31708F0E0E0132F1F1B21E09A
:106C0000311708F020E0E22B4B2F69969FAD699772
:106C1000491B31E0B41708F030E0B42FBE1B21E06F
:106C20004B1708F020E0322B502F6A96AFAD6A97D1
:106C30005A1B41E0051708F040E0052F031B21E037
:106C4000501708F020E0422B6F966FAD6F976B9650
:106C5000EFAD6B976E1B31E06F96FFAD6F97F61738
:106C600008F030E0962F941B21E0691708F020E02F
:106C7000322BA0967FADA0976C962FAD6C97721BB0
:106C800041E0A0968FADA097871708F040E0A72FAE
:106C9000A31B21E07A1708F020E0422BA1968FADCC
:106CA000A1976D96EFAD6D978E1B21E0A196FFAD7C
:106CB000A197F81708F020E0E82FE41B31E08E17C9
:106CC00008F030E0232BA296FFADA2976E963FAD61
:106CD0006E97F31BF21B232C280C31E0231408F0D1
:106CE00030E0812F890D41E0811708F040E0380F36
:106CF00051E0381708F050E0452B8B2F8A0D51E0FA
:106D00008B1708F050E0480F61E0481708F060E08A
:106D1000562B202F2B0D81E0201708F080E0520F1A
:106D200061E0521708F060E0682B690F71E06917A5
:106D300008F070E07A0F81E07A1708F080E08E0F9B
:106D400091E08E1708F090E0222D9F0F03E00E9443
:106D50009A59298F3A8F4B8F5C8F6D8F7E8F8F8FD3
:106D600098A3ED8CFE8C0F8D18A180911B01909142
:106D70001C01892BC9F480919C0790919D07009775
:106D800099F0A301920177FE07C022273327A901BA
:106D90002419350946095709A0E0B0E08217930786
:106DA000A407B5070CF459C48701F89480917F0BB0
:106DB0009091800BA091810BB091820B840D951D59
:106DC000A61DB71D80937F0B9093800BA093810B22
:106DD000B093820B80917D0B90917E0B8E0D9F1D49
:106DE00090937E0B80937D0B80917D0B90917E0B19
:106DF00097FF2AC080917F0B9091800BA091810B0F
:106E0000B091820B181619061A061B06ECF4809135
:106E10007F0B9091800BA091810BB091820B019719
:106E2000A109B10980937F0B9093800BA093810BF4
:106E3000B093820B80917D0B90917E0B88519C4F7B
:106E400090937E0B80937D0B80917F0B9091800BB4
:106E5000A091810BB091820B80938B0790938C074C
:106E6000A0938D07B0938E0780917D0B90917E0B40
:106E70009093920780939107789477FE0AC010163A
:106E800011063CF40894411C511C611C711C085EE5
:106E90001340D301C20180509048AF4FBF4F805084
:106EA0009040A140B04038F08FEF9FE79093740777
:106EB0008093730704C05092740740927307109335
:106EC00076070093750780917C09882361F1C301DF
:106ED000B20128EE33E040E050E00E9413619B01D4
:106EE000AC01C801AA2797FDA095BA2F820F931F66
:106EF000A41FB51FB7FD04C0B801620F731F0AC0FD
:106F0000C301B20128E13CEF4FEF5FEF0E94136134
:106F1000601B710B70937B0960937A096D5471400B
:106F200014F081E001C082E080937C0990C383303B
:106F300009F0E9C0292F287380917409909175098F
:106F40000197F1F550900601522A40900701E09018
:106F50008B07F0908C0700918D0710918E0780E8C9
:106F60009EE7AAEAB3E8E80EF91E0A1F1B1F60910C
:106F700091077091920780E090E00E9445313B01BB
:106F80004C01A0908707B0908807C0908907D090E7
:106F90008A0780E89EE7AAEAB3E8A80EB91ECA1ECF
:106FA000DB1E60918F077091900780E090E00E9457
:106FB000453165966CAF7DAF8EAF9FAF659713C0BF
:106FC00030EC532E522A65961CAE1DAE1EAE1FAE7F
:106FD0006597662477244301AA24BB246501EE2427
:106FE000FF24870144248AE290E00E949515852DB4
:106FF00084600E94C314842D0E94C3148BA10E943C
:10700000C31486EF0E94C31460E070E080E090E05B
:107010000E94E11460E070E080E090E00E94E114E2
:107020000E948E32C801B7010E94E114C401B3016D
:107030000E94E1148091740990917509019799F467
:10704000CE0181968C01085D1F4F20E3E22EF12CCA
:10705000E80EF91ED8018D918D010E94C3140E1502
:107060001F05C1F70CC060E070E080E090E00E9476
:10707000E11460E070E080E090E00E94E114C6015D
:10708000B5010E94E11465966CAD7DAD8EAD9FADEE
:1070900065970E94E1148091740990917509019798
:1070A00039F0EE24FF248701AA24BB2465011EC009
:1070B000F894E0907F0BF090800B0091810B109181
:1070C000820B80E89EE7AAEAB3E8E80EF91E0A1FE1
:1070D0001B1F60917D0B70917E0B882777FD80953B
:1070E000982F0E9445315B016C017894C801B7016B
:1070F0000E94E114C601B5010E94E11480E390E012
:107100000E940726ABC2853009F0A7C280916409AE
:107110008770813009F0A1C2892F807C809306019D
:107120009AA1803C09F499C2992309F496C290313E
:1071300009F493C29F5F909307016DA17EA18FA177
:1071400098A50E94E83D60937B0770937C0780932D
:107150007D0790937E0769A57AA58BA59CA50E94C3
:10716000E83D60937F077093800780938107909339
:107170008207FE01E05BFF4FD080FE01E15BFF4F25
:10718000C080FE01E25BFF4FA080FE01E35BFF4F8A
:1071900010813D2DD9822C2DCA829A2DAB82812F50
:1071A0001C83FE01E45BFF4FD080FE01E55BFF4FD7
:1071B000C080FE01E65BFF4FA080FE01E75BFF4F52
:1071C0001081DD82CE82AF821887032FF22EE92E46
:1071D000B82E832F822B892B8B298D298C298A29E4
:1071E000812B09F43AC2F89480917F0B9091800B27
:1071F000A091810BB091820B80589148A545BC4766
:107200008D839E83AF83B88760917D0B70917E0BD9
:10721000882777FD8095982F0E94453169837A836E
:107220008B839C83789489812A813B814C815D8109
:10723000AE81BF819884F02FF81B91E00F1708F002
:1072400090E08F2D821B21E0F81608F020E0E82F57
:10725000E91B91E08E1708F090E0292B8E2D831BFF
:1072600031E0E81608F030E0782F721B91E08717C4
:1072700008F090E0392B8B2D841B21E0B81608F024
:1072800020E0682F631B91E0861708F090E0292B1F
:107290008D2D851B31E0D81608F030E0582F521B99
:1072A00091E0851708F090E0392B8C2D8A1B21E0A6
:1072B000C81608F020E0482F431B91E0841708F01F
:1072C00090E0292B8A2D8B1B91E0A81608F090E006
:1072D000382F321B21E0831708F020E0922B191978
:1072E000191BF983EA837B836C835D834E833F8321
:1072F00018874D805E806F80788489819A81AB8108
:10730000BC814C015D01CC24DD2476019C01A501EA
:1073100060E070E080E090E002E00E949A59122F55
:10732000232EA3964FAFA397A4965FAFA497A596DD
:107330006FAFA597A6967FAFA697A7968FAFA79793
:10734000A8969FAFA89705E00E949A59A32FB42F43
:10735000052FA9966FAFA997AA967FAFAA97AB966C
:107360008FAFAB97AC969FAFAC97322E311AF1E04E
:10737000231508F0F0E03A2F3219E1E0A31708F0E6
:10738000E0E0132F1F1B21E0311708F020E0E22B73
:107390004B2FA3969FADA397491B31E0B41708F07C
:1073A00030E0B42FBE1B21E04B1708F020E0322B59
:1073B000502FA496AFADA4975A1B41E0051708F0D3
:1073C00040E0052F031B21E0501708F020E0422B7E
:1073D000A9966FADA997A596EFADA5976E1B31E065
:1073E000A996FFADA997F61708F030E0962F941BE9
:1073F00021E0691708F020E0322BAA967FADAA970A
:10740000A6962FADA697721B41E0AA968FADAA97BC
:10741000871708F040E0A72FA31B21E07A1708F098
:1074200020E0422BAB968FADAB97A796EFADA79719
:107430008E1B21E0AB96FFADAB97F81708F020E06C
:10744000E82FE41B31E08E1708F030E0232BAC96D8
:10745000FFADAC97A8963FADA897F31BF21B232C6A
:10746000280C31E0231408F030E0812F890D41E031
:10747000811708F040E0380F51E0381708F050E06D
:10748000452B8B2F8A0D51E08B1708F050E0480FE9
:1074900061E0481708F060E0562B202F2B0D81E0AB
:1074A000201708F080E0520F61E0521708F060E00A
:1074B000682B690F71E0691708F070E07A0F81E0BE
:1074C0007A1708F080E08E0F91E08E1708F090E0B8
:1074D000222D9F0F03E00E949A5929873A874B87F4
:1074E0005C876D877E878F87988BED84FE840F8500
:1074F000188980911B0190911C01892BC9F48091FE
:107500009C0790919D07009799F0A301920177FE47
:1075100007C022273327A90124193509460957092D
:10752000A0E0B0E082179307A407B5070CF495C05C
:107530009701F89480917F0B9091800BA091810B23
:10754000B091820B840D951DA61DB71D80937F0BF6
:107550009093800BA093810BB093820B80917D0B55
:1075600090917E0B8E0D9F1D90937E0B80937D0BD3
:1075700080917D0B90917E0B97FF2AC080917F0BAD
:107580009091800BA091810BB091820B1816190677
:107590001A061B06ECF480917F0B9091800BA09152
:1075A000810BB091820B0197A109B10980937F0BE8
:1075B0009093800BA093810BB093820B80917D0BF5
:1075C00090917E0B88519C4F90937E0B80937D0B06
:1075D00080917F0B9091800BA091810BB091820BD9
:1075E00080938B0790938C07A0938D07B0938E07A1
:1075F00080917D0B90917E0B9093920780939107E1
:10760000789477FE0AC0121613063CF40894411CC5
:10761000511C611C711C285E3340D301C201805093
:107620009048AF4FBF4F80509040A140B04038F0DD
:107630008FEF9FE7909374078093730704C0509275
:10764000740740927307309376072093750781E0A3
:1076500090E09093860B8093850B80E0C559DF4FB7
:10766000E2E10C94AB618091740990917509892BCA
:1076700011F480E008958AE290E00E949515F89454
:1076800060917F0B7091800B8091810B9091820BA8
:1076900078946058714885459C470E94E11484E0C5
:1076A00090E00E9407260895DB01982F92959F7025
:1076B0002CE531E0F901E90FF11DE491EC938F70B5
:1076C000280F311DF901849111968C931197129610
:1076D0001C921297CB010895DB01292F22952F7060
:1076E0004CE551E0FA01E20FF11DE491EC939F703B
:1076F000FA01E90FF11DE4911196EC931197982F7F
:1077000092959F70FA01E90FF11DE4911296EC93A6
:1077100012978F70480F511DFA01849113968C9324
:10772000139714961C921497CB010895DA01292F10
:1077300022952F704CE551E0FA01E20FF11DE49122
:10774000EC939F70FA01E90FF11DE4911196EC930F
:107750001197982F92959F70FA01E90FF11DE4910E
:107760001296EC9312978F70FA01E80FF11DE491D5
:107770001396EC931397872F82958F70FA01E80F79
:10778000F11DE4911496EC9314977F70FA01E70FC2
:10779000F11DE4911596EC931597862F82958F70C5
:1077A000FA01E80FF11DE4911696EC9316976F70AD
:1077B000460F511DFA01849117968C9317971896CE
:1077C0001C921897CD010895282FDB0164E60E94D2
:1077D0003261392F822F0E943261805DFD018193D9
:1077E000832F6AE00E943261805D11968C9311971D
:1077F000832F0E943261905D91831282CD010895A2
:10780000A0E0B0E0E6E0FCE30C949A61482FF92E8A
:10781000E62ED72E862F972F9C01E901E0E1F7E2B3
:1078200000E010E0842F9F2DBF010E943E61262FB3
:10783000842F9F2DBF010E943E61482FF92E205DAD
:107840002993CF016AE070E00E943E61FB010F5F67
:107850001F4F0430110531F7405D488319828E2D8A
:107860009D2DCDB7DEB7E7E00C94B661A0E0B0E0A7
:10787000ECE3FCE30C949261062F772E4C01642E0E
:10788000552E842F952F9C01E901C12C8AECD82E0E
:107890008AE9E82E8BE3F82EAA24BB24602F772DEB
:1078A000C401A70196010E945261122F602F772D0B
:1078B000C401A70196010E945261062F772E4C0148
:1078C000105D1993C701B6012AE030E040E050E0B6
:1078D0000E945261C901DA016C017D010894A11C6A
:1078E000B11C89E0A816B104C9F6005D08831982AD
:1078F000862D952DCDB7DEB7EFE00C94AE61EF92FB
:10790000FF920F931F938B019C01F42EE52E97FDA0
:1079100004C0842F952FFC010CC030952095109544
:1079200001951F4F2F4F3F4F842F952FFC018DE264
:107930008193C901B801AF010E94363C8F2D9E2D65
:107940001F910F91FF90EF9008951F93CF93DF93B6
:10795000EC0120E030E040E050E01881812F8053BE
:107960008A30C8F4CA01B9012AE030E040E050E0B2
:107970000E9413619B01AC01812F992787FD90958F
:10798000C097AA2797FDA095BA2F280F391F4A1F25
:107990005B1F2196E2CF203080E0380781E0480766
:1079A00080E0580720F02FEF3FEF40E050E0C901A2
:1079B000DF91CF911F910895982F8154863010F454
:1079C00087E307C0892F8156863010F487E501C010
:1079D00080E3981B892F0895FF920F931F938C01CA
:1079E000FC0180810E94DC3CF82EF29490EFF92299
:1079F000F80181810E94DC3C8F708F291F910F91CB
:107A0000FF900895EF92FF920F931F938C01FC015A
:107A100080810E94DC3CF82EF29430EFF322F801D2
:107A200081810E94DC3C8F70F82AF80182810E94DB
:107A3000DC3CE82EE29420EFE222F80183810E94F0
:107A4000DC3C8F708E299F2D1F910F91FF90EF903E
:107A50000895CF92DF92EF92FF920F931F938C01C4
:107A6000FC0180810E94DC3CC82EC29470EFC722CA
:107A7000F80181810E94DC3C8F70C82AF801828164
:107A80000E94DC3CD82ED29460EFD622F80183818C
:107A90000E94DC3C8F70D82AF80184810E94DC3C73
:107AA000F82EF29450EFF522F80185810E94DC3C1B
:107AB0008F70F82AF80186810E94DC3CE82EE2945F
:107AC00040EFE422F80187810E94DC3C8F708E2910
:107AD000682F7F2D8D2D9C2D1F910F91FF90EF9082
:107AE000DF90CF900895EF92FF920F931F938091B4
:107AF0007E0190917F01A0918001B09181017C0174
:107B00008D012BE0EE0CFF1C001F111F2A95D1F7F1
:107B1000E826F9260A271B2780918201909183018C
:107B2000A0918401B091850180937E0190937F01A3
:107B3000A0938001B093810180918601909187018B
:107B4000A0918801B0918901809382019093830173
:107B5000A0938401B093850180918A0190918B015B
:107B6000A0918C01B0918D01809386019093870143
:107B7000A0938801B09389019C01AD01F3E1569572
:107B8000479537952795FA95D1F7282739274A271A
:107B90005B272E253F2540275127EF2CF02E012F64
:107BA00011272E253F254027512720938A01309306
:107BB0008B0140938C0150938D01B901CA011F9133
:107BC0000F91FF90EF900895282F892F922F0895FD
:107BD000362F272F692F782FC9010895A0E2B0E032
:107BE000E4EFFDE30C9495619C015B018E010F5F56
:107BF0001F4FC801B9010E946F62CC24DD247601B9
:107C0000980140E1842E912C8C0E9D1EF8018081FC
:107C10008E3291F41082C9010E94A53CA0E0B0E030
:107C20008C299D29AE29BF29CC24D82EE92EFA2EE5
:107C300098012F5F3F4F2BC08823E9F4CE010196B6
:107C40000817190731F4F50110821182128213828C
:107C500010C0F8011082C9010E94A53CA0E0B0E06C
:107C60008C299D29AE29BF29F50180839183A283A8
:107C7000B38381E013C0992787FD9095C0970A9739
:107C800030F0F501108211821282138206C00815AD
:107C9000190519F00F5F1F4FB9CF80E0A096ECE0F7
:107CA0000C94B161CF92DF92EF92FF920F931F93EA
:107CB0006B01E82E8A01892FBA010E94E43B5EE243
:107CC000F52EF801F382B8016C5F7F4F8E2D0E9474
:107CD000E43BF801F782B801685F7F4F8D2D0E9469
:107CE000E43BF801F386B801645F7F4F8C2D0E945E
:107CF000E43BC8011F910F91FF90EF90DF90CF9070
:107D00000895CF92DF92EF92FF920F931F936B0132
:107D10000E94441D7B018C01C6010E94441D9B01F1
:107D2000AC012E193F09400B510BB901CA011F913B
:107D30000F91FF90EF90DF90CF900895A4E0B0E016
:107D4000E4EAFEE30C949D61162F072F0E94441D68
:107D500020917701309178014091790150917A0119
:107D6000260F371F481F591F29833A834B835C8393
:107D7000CE0101960E949C1DAC01009711F480E099
:107D80000BC0812F902F9C01D901FA0182E1019053
:107D90000D928150E1F781E02496E4E00C94B96102
:107DA000A4E0B0E0E6EDFEE30C949961D62EC72E78
:107DB00079018A010E94441D6E197F09800B910B85
:107DC00069837A838B839C83CE0101960E949C1DDC
:107DD000AC01009711F480E00BC08D2D9C2D9C010F
:107DE000D901FA0182E101900D928150E1F781E021
:107DF0002496E8E00C94B561EF92FF920F931F93E5
:107E0000E82EF62E8A01FA940E94271BF80180833F
:107E1000813131F48E2D8F5FF81660F480E00AC056
:107E2000823111F08E2D06C0EE2011F48F2D02C08C
:107E30008E2D81501F910F91FF90EF900895A0E03B
:107E4000B0E0E5E2FFE30C949061C82E362E7A0193
:107E5000B22EE8010E94C419EB2DFF27E7FDF09533
:107E6000EE0DFF1D1082F7019081892F80538A301B
:107E700010F4182F08C0892F8154863010F010E0BC
:107E800002C0192F1753A8951B9BFDCF81E00E94BC
:107E90007719219711F08AE001C080E1012F1127A5
:107EA00007FD1095DC2CC0E0D0E04B2C552447FC9E
:107EB0005094882E992487FC90943401089461088A
:107EC00071085701AC0EBD1E8D2D632D0E948B19BC
:107ED0000A30110518F4802F805D02C0802F895C64
:107EE0000E945B190E946F190E94271B813141F487
:107EF0000F5F1F4F081519054CF000E010E006C099
:107F0000823179F40150104017FD83010A301105C8
:107F100018F4802F805D02C0802F895CF50180837A
:107F2000D0CF833151F52196D394F701EC0FFD1F8B
:107F30008081992787FD90950E94C661892B11F455
:107F40002196D394C415D5051CF0DC2CC0E0D0E0FC
:107F5000F701EC0FFD1FE0818E2F80538A3040F037
:107F60008E2F8154863010F080E002C08E2F875310
:107F7000082F112707FD1095A4CF843119F401E0D3
:107F800010E005C0893109F09CCF00E010E080E0EE
:107F90000E947719C801CDB7DEB7E1E10C94AC615E
:107FA0008091910B8130C1F580918B0B90918C0B5E
:107FB000A0918D0BB0918E0B0196A11DB11D8093E8
:107FC0008B0B90938C0BA0938D0BB0938E0B8091A9
:107FD0008B0B90918C0BA0918D0BB0918E0B80939D
:107FE0008B0790938C07A0938D07B0938E07809397
:107FF0007F0B9093800BA093810BB093820B109218
:1080000092071092910781E090E09093860B809305
:10801000850B1092910B3EC080918F0B823099F0AE
:1080200080917F0B9091800BA091810BB091820B7E
:108030000196A11DB11D80937F0B9093800BA0939F
:10804000810BB093820B809164098770823031F587
:10805000209165093091660921153105D9F080918B
:10806000890B90918A0B019690938A0B8093890BD0
:108070008091890B90918A0B8217930778F089E0A1
:1080800080937D0180917C01843041F083E0809376
:108090007C0104C010928A0B1092890B80917C01A4
:1080A0008130C1F48091670990916809892B91F022
:1080B0008091870B9091880B01979093880B809308
:1080C000870B8091870B9091880B892B19F482E0A4
:1080D00080937C0181E090E09093840B8093830BEC
:1080E00008951F920F920FB60F9211242F933F9372
:1080F0004F935F936F937F938F939F93AF93BF93B0
:10810000EF93FF9382E083BD1092B2001CBA1DBAB8
:1081100088EC80937B018091910B8230C1F41092A6
:108120007E0B10927D0B109292071092910781E0C6
:1081300090E09093860B8093850B10928A0B10929F
:10814000890B1092910B9093840B8093830B8091F9
:10815000910B813091F4809164098770833039F4F8
:1081600084E690E090937E0B80937D0B04C0109288
:108170007E0B10927D0B0E94D03F8AE08093900B83
:10818000FF91EF91BF91AF919F918F917F916F91EF
:108190005F914F913F912F910F900FBE0F901F90C5
:1081A00018951F920F920FB60F9211240F900FBEC9
:1081B0000F901F9018951F920F920FB60F921124D7
:1081C0000F900FBE0F901F9018951F920F920FB631
:1081D0000F9211242F933F934F935F936F937F934D
:1081E0008F939F93AF93BF93EF93FF9380917D0BFA
:1081F00090917E0B019690937E0B80937D0B8091E6
:10820000910B8230C9F410927E0B10927D0B10926C
:1082100092071092910781E090E09093860B8093F3
:10822000850B10928A0B1092890B1092910B9093F0
:10823000840B8093830B0DC080917D0B90917E0BFE
:10824000885E9340BCF010927E0B10927D0B0E94D2
:10825000D03F8091900B882331F08091900B81501A
:108260008093900B07C080917D01873019F486E0E0
:1082700080937D01FF91EF91BF91AF919F918F917D
:108280007F916F915F914F913F912F910F900FBE12
:108290000F901F9018951F920F920FB60F921124F6
:1082A0008F939F938091BA029091BB020196909315
:1082B000BB028093BA0280917B01882359F08091A0
:1082C0007B01815080937B0180917B01882311F495
:1082D00081E08DBB9F918F910F900FBE0F901F90EB
:1082E00018951F920F920FB60F9211248F939F93A0
:1082F000EF93FF938091C0009091C6008C7181F440
:1083000080918603E82FF0E0EB5FFC4F90838F5F56
:108310008F7780938603809187038F5F8093870395
:10832000FF91EF919F918F910F900FBE0F901F9033
:1083300018951F920F920FB60F9211242F938F93BF
:108340009F93EF93FF93209102032223B9F0909122
:108350000103E92FF0E0EF53FD4F80818093C600C9
:108360009F5F90930103822F8150809302038823A3
:1083700029F48091C1008F7D8093C100FF91EF911E
:108380009F918F912F910F900FBE0F901F90189576
:108390001F920F920FB60F9211248F9380910203B8
:1083A000882349F48091C1008F7B8093C100109293
:1083B0000403109203038F910F900FBE0F901F9034
:1083C0001895CF93DF93EC0163E37BE044E050E04A
:1083D0000E940662892B11F481E017C0CE016FE282
:1083E0007BE043E050E00E940662892B11F482E0BA
:1083F0000CC0CE0168E27BE046E050E00E940662DD
:10840000892B11F483E001C080E0DF91CF910895C2
:10841000CF93DF93019719F0C0E0D0E005C083E56A
:108420009DE00E94C717EC0187E39DE00E94C717FB
:108430009E01280F391FC901DF91CF910895A0E057
:10844000B0E0E5E2F2E40C9491613B01E82FFF27F4
:10845000E7FDF095EE0FFF1FED53F84F4590549058
:1084600086EF9DE00E94C7174C01C2010E94C7170A
:10847000EC0188ED9DE00E94C7175C01C2010E94DB
:10848000C7176C018AEB9DE00E94C7177C01C201EF
:108490000E94C7178C0186EA9DE00E94C717C80D8D
:1084A000D91DCA0DDB1DCC0DDD1DCE0DDF1DC00F8E
:1084B000D11FC80FD91F81E068167104A9F486E99D
:1084C0009DE00E94C7177C01C2010E94C7178C0162
:1084D0008BE79DE00E94C7179701200F311F2C0FDB
:1084E0003D1F280F391F07C086E79DE00E94C71770
:1084F0009C012C0F3D1FC901CDB7DEB7E0E10C9404
:10850000AD61EF92FF920F931F93182F86E390E0D7
:108510000E9495158EED91E00E94C7177C01E12F16
:10852000FF27E7FDF095EE0FFF1FE35CF74F859106
:1085300094910E94C7178C018CE09EE00E94C7179F
:108540000E0D1F1D080F191FC8011F910F91FF90DD
:10855000EF900895A0E0B0E0E0EBF2E40C949761B6
:10856000082F86E390E00E9495158EED91E00E9421
:10857000C7175C01C02FDD27C7FDD095CC0FDD1FCD
:10858000FE01E35CF74F859194910E94C7178C011F
:1085900088E49EE00E94C7176C01FE01ED53F84F7E
:1085A000859194910E94C7177C018AE39EE00E9406
:1085B000C7170A0D1B1D0C0D1D1D0E0D1F1D080FCD
:1085C000191FC801CDB7DEB7EAE00C94B361AF92D2
:1085D000BF92CF92DF92EF92FF920F931F938C0185
:1085E000F62EE72E89ED9CE00E94C7175C01C801BA
:1085F0000E94C7178C018FEC9CE00E94C7176C018A
:10860000EF2DFE2DDF010D900020E9F71197AE1B35
:10861000BF0B8F2D9E2DBD010E94FA147C0184ECAE
:108620009CE00E94C7170A0D1B1D0C0D1D1D0E0D91
:108630001F1D080F191FC8011F910F91FF90EF9088
:10864000DF90CF90BF90AF900895A4E0B0E0EBE250
:10865000F3E40C949F61BE016F5F7F4F0E94E43B87
:10866000CE01029662E070E00E94FA142496E2E0E5
:108670000C94BB61A8E0B0E0E0E4F3E40C949361F7
:108680007C01FC0180819181BE016F5F7F4F0E9460
:10869000003CCE01029664E070E00E94FA143C01B6
:1086A0008FE20E94C314F70182810E9425438C014E
:1086B0008FE20E94C314F70183810E9425434C017D
:1086C00080E20E94C314F70184810E9425435C016B
:1086D0008AE30E94C314F70185810E9425436C013F
:1086E0008AE30E94C314F70186810E942543080D86
:1086F000191D0B5F1F4F0A0D1B1D0C0D1D1D080FB3
:10870000191F060D171DC8012896EEE00C94AF61E5
:10871000A8E0B0E0EEE8F3E40C948F616C0180E334
:108720009DE00E94C7179E838D83F6018081918111
:108730000E94C7178C0182E19DE00E94C7179887AD
:108740008F83F601828193810E94C7171C0189E003
:108750009DE00E94C7172C01F60184817E010894D8
:10876000E11CF11CB7010E94E43BF70101900020DD
:10877000E9F73197EE19FF09BF010E94FA143C0195
:108780008BEF9CE00E94C7174C01F6018581B70171
:108790000E94E43BF70101900020E9F73197EE19C0
:1087A000FF09BF010E94FA145C0181EF9CE00E9466
:1087B000C7177C01F60186819781FC01DF010D90CE
:1087C0000020E9F71197AE1BBF0BBD010E94FA1400
:1087D0002D813E81020F131FEF81F8850E0F1F1FA1
:1087E000020D131D040D151D060D171D080D191D75
:1087F0000A0D1B1D0E0D1F1D080F191FC8012896FD
:10880000E2E10C94AB61A8E2B0E0E9E0F4E40C949E
:108810009B61082F112707FD1095000F111FF8010C
:10882000E75DFB4F85919491F801E45BFE4F459124
:10883000549139E0E32EF12CEC0EFD1EB7010E949D
:10884000521BF801EF5DFB4F859194919A838983C8
:10885000F801E750FC4F859194919C838B8381E2D2
:108860008D838FE18E83F886EF82CE0101960E9480
:108870008843A896E6E00C94B761A8E1B0E0E3E491
:10888000F4E40C949B61E82EFF24E7FCF09487014C
:10889000000F111FF801ED56FC4F8591949101C016
:1088A000A895F999FDCF0E94A3629B01AC012F3FCF
:1088B0008FEF38078FEF48078FEF580759F4F7010C
:1088C000EE0FFF1FEE0FFF1FE356FC4F2591359172
:1088D00045915491F801ED51FC4F859194919A8303
:1088E0008983F801E757FC4F859194919C838B8392
:1088F00082E18D838FE08E83CA01B901AE01475FAB
:108900005F4F0E94523E98878F83CE0101960E944E
:1089100088436896E6E00C94B761A0E0B0E0E3E934
:10892000F4E40C9497615C0180E00E94AA426C011F
:1089300080E00E943D44EC0181E00E943D447C01C6
:1089400082E00E943D448C0183E00E943D44CC0DB6
:10895000DD1DCE0DDF1DC00FD11FC80FD91F81E057
:10896000A816B10419F48DE093E002C085E493E009
:108970000E94C717C80FD91F81E090E00E940842EB
:108980006091E5047091E604C80FD91F88E1AE013B
:108990000E944622CDB7DEB7EAE00C94B361AAE9A3
:1089A000B0E0E5EDF4E40C948F619C01880F991F11
:1089B000BC01F3E0660F771FFA95E1F7680F791FA6
:1089C00061547B4F7093E6046093E504F901E5512F
:1089D000F94FE081E13009F070C6232B29F0E7EE72
:1089E0008E2EE5E09E2E04C077EE872E74E0972E43
:1089F000C4016AE879E00E941462FC01108263EC11
:108A0000E62E67E0F62E00E0F70165917491C4014F
:108A100046E050E00E940662892B09F455C00F5FC2
:108A200022E030E0E20EF31E063071F786E390E0BC
:108A30000E9495158EED91E00E94C7172C018EEAD9
:108A400099E00E94C717480E591E882499248EE980
:108A500099E00E94C7175C01F401ED53F84F85912E
:108A600094910E94C7178C018AE999E00E94C71768
:108A70006C01F401E35CF74F859194910E94C71754
:108A80007C0181E999E00E94C7170A0D1B1D0C0D9E
:108A90001D1D0E0D1F1D080F191F400E511E42E017
:108AA00050E0840E951E5CE08516910481F680E00E
:108AB00090E00E9408426091E5047091E604480E3F
:108AC000591E88E1A2010DC657E0452E512C480CD5
:108AD000591C002309F043C0D40117968C918823B8
:108AE00019F480E090E038C000E010E06E010894D6
:108AF000C11CD11C46E0842E912C800E911EF401E5
:108B0000E757FC4F65917491C2010E9414627C0189
:108B1000009701F10396B6010E94EE3D813079F491
:108B2000F401ED56FC4F8591949101C0A895F999F7
:108B3000FDCF49815A816B817C810E94D16208946A
:108B4000E108F108F701108202501040FFEF083FE2
:108B50001F0781F681E090E00E948D44C4C501307A
:108B600009F081C0D2018C91882319F488249924BA
:108B700059C0DE011C96EEE8F1E088E001900D920C
:108B80008150E1F732E1832E912C8C0E9D1E00E086
:108B900010E02CE3C22ED12CCC0EDD1E90E2B92EBB
:108BA00086E0282E312C200E311EF101E750FC4FBB
:108BB00065917491C2010E9414627C01009779F161
:108BC000F6012B2D11922A95E9F7BC016D5F7F4FBD
:108BD000C6010E946F62D4018D919C91B6010E94E2
:108BE0006F62F101E75DFB4F6591749101C0A8953B
:108BF000F999FDCFC60140E250E00E94AF620894AF
:108C0000E108F108F7011082025010402EEF3FEF0B
:108C1000820E931E3FEF083F130709F0C1CFB1E06A
:108C20008B2E912C81E00E94AA426C0180E00E9470
:108C300003442C0181E00E9403447C0182E00E94F5
:108C400003448C0183E00E9403444C0C5D1C4E0CD9
:108C50005F1C400E511E480E591E41E084169104BF
:108C600009F07FC07BC0023009F08FC0D2018C9127
:108C7000882319F48824992445C0C20167EC79E05F
:108C80000E9414627C010097D1F105960E94A53CD8
:108C900090939807809397078F5F9F4F31F41092BE
:108CA00098071092970701C0A895F999FDCF609198
:108CB00097077091980784EC90E00E94DD62089419
:108CC000E108F108F7011082C20164EC79E00E942A
:108CD00014620097A1F00396BE016F5F7F4F0E9460
:108CE000EE3D813061F401C0A895F999FDCF49812D
:108CF0005A816B817C8180EC90E00E94D162A1E07E
:108D00008A2E912C82E00E94AA426C0184E00E948B
:108D10003D442C018CEC99E00E94C7177C018E0128
:108D20000C5E1F4F8091970790919807B8010E94A1
:108D3000003CF80101900020E9F73197E01BF10BAE
:108D4000C801BF010E94FA144C0C5D1C4E0C5F1C44
:108D5000480E591EF1E08F16910419F48DE093E04E
:108D600002C085E493E00E94C7177C01E40CF51C67
:108D700081E090E00E9408426091E5047091E60471
:108D8000E80EF91E88E1A701ACC4033009F04FC119
:108D9000C2010E94E141813019F4F8E0FF2E05C0C4
:108DA000823011F40E944A4FFF2483E00E948142E6
:108DB0008C0189E39AE00E94C7176091E5047091E5
:108DC000E604080F191F88E1A8010E9446228823A3
:108DD00009F089C486E390E00E9495156F2CAA24BF
:108DE000BB24ECE22E2E312C2C0E3D1E2F2D285FA5
:108DF000C656DF4F2883CA59D040E62DF0E074E014
:108E0000EE0FFF1F7A95E1F7DE015C96E358F64F0F
:108E100080E101900D928150E1F7DBA04C8C5D8CDC
:108E20003E8DCE57DF4F3883C258D0404F8DCF573D
:108E3000DF4F4883C158D04058A1C058DF4F5883F6
:108E4000C058D04079A0CAA08CA09DA08EA19FA19F
:108E5000C258DF4F99838883CE57D04080E19BE092
:108E60000E94C7178C016394862D0E9425437C01C4
:108E700086E09BE00E94C717E00EF11EE80EF91E87
:108E80008D2D81508330D8F45E824D82CE57DF4FD6
:108E90009881C258D0409F83CF57DF4FA881C158D7
:108EA000D040A887C058DF4FB881C058D040B9879C
:108EB0007A86CB86CE0105960E943A4304C08FEF96
:108EC0009AE00E94C717E80EF91E85EF9AE00E940B
:108ED000C7172701480E591EE2E0DE1661F486EE40
:108EE0009AE00E94C7177C0189ED9AE00E94C7179B
:108EF000E80EF91E77C0F1E0DF1609F06EC021E937
:108F000082162EE7920644F08CEC9AE00E94C71776
:108F10007C01E40CF51C5AC097FC02C08BE201C036
:108F20008DE20E94C314C40197FE03C09095819501
:108F30009F4FB1010E94003CF10101900020E9F730
:108F40003197E219F309C101BF010E94FA144C01E3
:108F500087EC9AE00E94C7176C01C258DF4F488126
:108F60005981CE57D04057FD02C08BE201C08DE23F
:108F70000E94C314C258DF4F88819981CE57D040D8
:108F800097FF03C0909581959F4FB1010E94003CCF
:108F9000F10101900020E9F7E219F3093397CE01BE
:108FA0008E96BF010E94FA148C0183EC9AE00E9415
:108FB000C71762E0E62EF12CE40CF51CE80CF91C56
:108FC000EC0CFD1CE00EF11EE80EF91E80EB9AE0A1
:108FD0000E94C717E80EF91E07C080EA9AE00E94B7
:108FE000C7177C01E40CF51C85E99AE00E94C717BD
:108FF000E80EF91EAE0CBF1CC656DF4F5881CA5989
:10900000D040651609F0F9CE6091E5047091E60450
:1090100088E1A5010E944622882309F064C386E303
:1090200090E00E94951583E060E070E098C1043004
:1090300009F09DC1C2010E94E141813039F488E00C
:10904000C856DF4F8883C859D0400DC0823019F40C
:109050000E943F4F03C0833009F4179AC856DF4F70
:109060001882C859D04084E00E9481428C0188E374
:109070009BE00E94C7176091E5047091E604080F19
:10908000191F88E1A8010E944622882309F02BC3FA
:1090900086E390E00E949515C956DF4F1882C759A4
:1090A000D040EE961FAE1EAEEE9754E1252E312C29
:1090B0002C0E3D1E8EEC9BE00E94C7178C01C956FA
:1090C000DF4FE881C759D040C856DF4F9881C85953
:1090D000D040E90FF0E044E0EE0FFF1F4A95E1F7C2
:1090E000CF018358954FDC011C962D913D914D91F8
:1090F0005C911F97CD56DF4F288339834A835B836A
:10910000C359D0401A96CC901A971B96BC91C7565B
:10911000DF4FB883C959D040DF01AB57B54FEC9052
:109120001196DC90DC0116966C91169715965C9161
:10913000DF01AF57B54F7C91DC0113964C9113972B
:10914000E158F54FE0812D913C9111971796FC90D5
:10915000FF2009F4CAC08F2D8150843028F48AEB97
:109160009BE00E94C7170BC03E832D83EF83488787
:1091700079875A876B87CE0105960E943A43080F7C
:10918000191F80EB9BE00E94C7172C01EF2DF0E028
:10919000EE0FFF1FEC5BF84F859194910E94C7176B
:1091A000400E511E480E591EB5E0FB1609F03FC097
:1091B0008AEA9BE00E94C7173C018E2D9D2DB101CC
:1091C0000E946C3BF10101900020E9F73197E21910
:1091D000F309C101BF010E94FA144C0184EA9BE02B
:1091E0000E94C7175C018C2DC756DF4F9881C95963
:1091F000D040B1010E946C3BF10101900020E9F7E1
:109200003197E219F309C101BF010E94FA146C0100
:109210008DE99BE00E94C7177C01CD56DF4F888106
:109220009981C359D040B1010E946C3B41C0EAE032
:10923000FE1621F0F7E0FF1609F05EC086E99BE01C
:109240000E94C7173C018E2DB1010E94543BF101D1
:1092500001900020E9F73197E219F309C101BF013C
:109260000E94FA144C018FE89BE00E94C7175C0132
:109270008C2DB1010E94543BF10101900020E9F7CF
:109280003197E219F309C101BF010E94FA146C0180
:1092900087E89BE00E94C7177C01CD56DF4F6881AD
:1092A00079818A819B81C359D040A1010E94963B5C
:1092B000F10101900020E9F73197E219F309C101AA
:1092C000BF010E94FA148C0189E20E94C314089421
:1092D000411C511C460C571C480C591C4A0C5B1C69
:1092E0004C0C5D1C4E0C5F1C05C081E79BE00E948E
:1092F000C7172C01400E511E86E69BE00E94C7173F
:10930000480E591EEE962EAD3FADEE97240D351D3D
:10931000EE963FAF2EAFEE97C956DF4F3881C75953
:10932000D0403F5FC956DF4F3883C759D0403830EF
:1093300009F0C0CE6091E5047091E60488E1EE96F4
:109340004EAD5FADEE970E944622882309F0CBC157
:1093500086E390E00E94951584E061E070E00E9451
:109360001F428C0181E090E00E94084298C10530C4
:1093700009F09EC185E00E948142CF56DF4F99835C
:109380008883C159D04086E99CE00E94C7178C01B0
:109390006091AA047091AB048091AC049091AD04EB
:1093A0002CE3E22EF12CEC0EFD1EA7010E94523E92
:1093B000BC018BE89CE00E94E742CD57DF4F9983C8
:1093C0008883C358D0406091AE047091AF048091FF
:1093D000B0049091B104A7010E94523EBC018FE7F6
:1093E0009CE00E94E742CB57DF4F99838883C558A2
:1093F000D0406091B2047091B3048091B404909114
:10940000B504A7010E94523EBC018FE69CE00E9479
:10941000E742C957DF4F99838883C758D04060918E
:109420005E0970915F098091600990916109A701BF
:109430000E94523EBC0184E69CE00E94E742C7576E
:10944000DF4F99838883C958D04087E59CE06EE45C
:1094500079E00E94E742C557DF4F99838883CB5854
:10946000D04080916409E82FF0E0E770F070EE0FD3
:10947000FF1FEB55F74F65917491C7010E94F6618C
:1094800088E49CE0B7010E94E742C357DF4F99830D
:109490008883CD58D04080917D01E82FF0E0EE0F19
:1094A000FF1FEA58F64F65917491C7010E94F6615B
:1094B0008CE39CE0B7010E94E742C157DF4F9983DC
:1094C0008883CF58D04080910001B7010E94543B5F
:1094D00080910101BE01625C7F4F0E94543BB70145
:1094E0006C5F7F4F809102010E94543B8DE2FE0130
:1094F000EE5BFF4F8083B701695F7F4F809103016F
:109500000E94543BB701675F7F4F809104010E9426
:10951000543BB701655F7F4F809105010E94543B2A
:10952000FE01E75BFF4F108280E39CE0B7010E94E1
:10953000E7421C0120911804822F6AE00E943261E8
:10954000805D8CAF822F0E943261905D9DAF1EAE18
:109550008EE19CE0B7010E94E7422C01C7016CE755
:1095600070E00E94F6618DE09CE0B7010E94E74246
:109570003C0180906D0990906E09A0906F09B090A9
:109580007009C501B4012CE330E040E050E00E94D6
:109590007461CA01B901A7010E947F3C7CE5C72E16
:1095A000D12CCC0EDD1EB7016B5F7F4FC6010E9430
:1095B0006F62C60167E07CE00E94E261C501B40110
:1095C0002CE330E040E050E00E947461DC01CB010C
:1095D000B7010E94003CC601BE01615C7F4F0E9442
:1095E0005062C60162E07CE00E94E26183EF9BE092
:1095F000B6010E94E7426C0186EE9BE00E94C7170D
:109600007C0181E090E00E940842CF56DF4F488104
:109610005981C159D040040F151FCD57DF4FA88184
:10962000B981C358D0400A0F1B1FCB57DF4FE881C9
:10963000F981C558D0400E0F1F1FC957DF4F288131
:109640003981C758D040020F131FC757DF4F4881D9
:109650005981C958D040040F151FC557DF4FA88145
:10966000B981CB58D0400A0F1B1FC357DF4FE88189
:10967000F981CD58D0400E0F1F1FC157DF4F2881F1
:109680003981CF58D040020F131F020D131D040D56
:10969000151D060D171D0C0D1D1D0E0D1F1D6091B6
:1096A000E5047091E604080F191F88E1A80119C0AC
:1096B0006091E5047091E60411C0E23079F486E32C
:1096C00090E00E9495158DE691E00E94C717AC01CD
:1096D0006091E5047091E60488E103C081E140E017
:1096E00050E00E944622C656DF4FE2E10C94AB6187
:1096F000682F88E046E753E10E94B4190895E82FE7
:10970000F0E0EE0FFF1FE65CFF4E4591549180E0C4
:1097100061E00E94B4190895E82FF0E0EE0FFF1FFA
:10972000E357F04F4591549180E060E00E94B419F6
:109730000895A0E1B0E0EFE9FBE40C949961E090BA
:109740006D09F0906E0900916F0910917009C801C0
:10975000B7012CE330E040E050E00E947461CA01A0
:10976000B9016E010894C11CD11CA6010E947F3C66
:1097700080E061E0AE014A5F5F4F0E94C419C801FA
:10978000B7012CE330E040E050E00E947461DC015E
:10979000CB01B6010E94003C8AE061E0AE014C5F63
:1097A0005F4F0E94C4196096E8E00C94B561A4E094
:1097B000B0E0EDEDFBE40C949761B82EA62E6A01A3
:1097C000FA0180817E010894E11CF11CB7010E941E
:1097D000E43B8E010E5F1F4F8B2D6A2DA8010E9466
:1097E000C4198AE30E945B19F6018181B7010E94C6
:1097F000E43BC8010E9462198AE30E945B19F601EA
:109800008281B7010E94E43BC8010E94621924963C
:10981000EAE00C94B361A3E0B0E0E1E1FCE40C9475
:109820009A61D82E7A018B0140348EE7580785E083
:10983000680780E0780738F088E06D2D4DE653E149
:109840000E94B4192EC0CB01BA0120E13EE040E0F5
:1098500050E00E9474612983C801B70120E13EE015
:1098600040E050E00E947461162F072FF82EE92E79
:109870002CE330E040E050E00E9474612A83612FC5
:10988000702F8F2D9E2D2CE330E040E050E00E94A1
:1098900074616B8388E06D2DAE014F5F5F4F0E9456
:1098A000D74B2396E7E00C94B6618091D5078130C1
:1098B00049F44091CE075091CF076091D007709145
:1098C000D1071BC08731E1F48091CA079091CB0783
:1098D000A091CC07B091CD078F5F9F4FAF4FBF4F87
:1098E00019F4EAE7F0E115C04091C2075091C307AF
:1098F0006091C4077091C50781E00E940B4C0895E8
:10990000883119F4E8E7F0E104C0893139F4E6E779
:10991000F0E14591549188E061E004C088E061E0A5
:1099200046E753E10E94B4190895A3E2B0E0EBE9E1
:10993000FCE40C949661082F0E948319093018F4F6
:10994000402F4F5C02C0402F49508FE060E00E94E2
:10995000CF19E02FF0E044E0EE0FFF1F4A95E1F74A
:10996000DE011496E358F54F80E101900D9281508D
:10997000E1F7DB849E81CF809884A984BA848D2D01
:109980008150843068F18D2D8550823248F534E164
:10999000E32EF12CEC0EFD1E892FB7010E94E43B53
:1099A0008E010B5E1F4F80E060E0A8010E94C41989
:1099B0008FE20E945B198C2DB7010E94E43BC80125
:1099C0000E94621980E20E945B199982AA82BB827E
:1099D00086E060E0AE014F5F5F4F0E94D74B06C04C
:1099E00080E060E042E553E10E94B419ED2DF0E023
:1099F000EE0FFF1FEC5FFC4E4591549180E061E05B
:109A00000E94B419A396EBE00C94B261A3E2B0E01B
:109A1000ECE0FDE40C949561182F0E9483198BE013
:109A20000E948C4BE12FF0E064E0EE0FFF1F6A957F
:109A3000E1F7DE011496E358F64F80E101900D92B4
:109A40008150E1F7DB84CE80BF8088849984AA842A
:109A500054E1E52EF12CEC0EFD1E812F8F5FB70136
:109A60000E94E43B8E010B5E1F4F8EE060E0A80178
:109A70000E94C41980E061E00E948B198D2D8150F5
:109A8000823068F58C2DB7010E94E43BC8010E942A
:109A900062198FE20E945B198B2DB7010E94E43B93
:109AA000C8010E94621980E20E945B1989829A8231
:109AB000AB8286E061E0AE014F5F5F4F0E94D74B03
:109AC00080E20E945B1982E0D81611F482E404C09F
:109AD00081E0D81651F482E50E945B1906C080E04F
:109AE00061E042E553E10E94B419A396ECE00C94C6
:109AF000B161A3E1B0E0EFE7FDE40C9493618091E4
:109B00007209E82FF0E0EE0FFF1FEC56FF4E659153
:109B10007491CE0108960E94F66160901D017090CC
:109B20001F0180902101A0902901B0902A0100918D
:109B30002501109126010F5F1F4F90902301809106
:109B4000270190912801FCE0CF2ED12CCC0EDD1EF8
:109B50008459984FB6010E94003CEDE0EE2EF12CA6
:109B6000EC0EFD1E80E060E0A7010E94C4198FE2A8
:109B70000E945B19802FB6010E94E43BC7010E943E
:109B800062198FE20E945B19892DB6010E94E43BA5
:109B9000C7010E94621980E20E945B198E010C5F6E
:109BA0001F4FAA0CBB1CAA0CBB1C8FE59EE0A80E85
:109BB000B91EC801B5010E94F661C8010E94621970
:109BC00080E20E945B1900916409077091F4809112
:109BD0000601803C11F481E415C0803411F489E45D
:109BE00011C0803811F484E40DC080917107805D4C
:109BF00009C0013011F482E505C0023011F08AE499
:109C000001C087E40E945B1989827A826B8280E0BE
:109C100061E0AE014F5F5F4F0E94D74B80E20E9430
:109C20005B19CE0108960E94621980E20E945B19BE
:109C3000023060F480910701BE016C5F7F4F0E948B
:109C4000E43BCE0105960E94621921C00230C9F49E
:109C500080916409887321F486E40E945B190FC027
:109C6000883011F482E503C0803189F48AE50E94CE
:109C70005B198091640986FF02C082E506C086E414
:109C800004C080E30E945B1981E30E945B19E091AC
:109C90007D01F0E0E558F14FE4918E2F0E945B19B1
:109CA0006396EEE00C94AF61A0E1B0E0EAE5FEE47B
:109CB0000C949961009162090E948319002319F4A0
:109CC0000E94794DD8C0013019F580E060E041E490
:109CD0000E94CF196091AA047091AB048091AC04EA
:109CE0009091AD048E010F5F1F4FA8010E94523E5C
:109CF0000E94621980E061E04DE40E94CF196091FA
:109D0000AE047091AF048091B0049091B10424C06E
:109D1000023041F580E060E047E40E94CF19609195
:109D2000B2047091B3048091B4049091B5048E0193
:109D30000F5F1F4FA8010E94523E0E94621980E0EF
:109D400061E044E40E94CF1960915E0970915F095F
:109D50008091600990916109A8010E94523E0E9481
:109D6000621989C0033079F581E00E948C4B8091A3
:109D700018046AE00E943261805D0E945B19809144
:109D800018046AE00E943261892F805D0E945B198D
:109D900083E00E947F4B04E0B0E0EB2EB1E0FB2EAD
:109DA0006E010894C11CD11CF70181917F01B6019D
:109DB0000E94543BAC01802F61E00E94C4190E5FE9
:109DC000003191F758C0043061F480E060E04EE467
:109DD00059E00E94C41984E00E947F4B0E94554CB8
:109DE0004AC0053091F586E00E948C4B8091640951
:109DF0008770823031F0813021F08091730988239F
:109E000091F188E060E046E753E10E94B41985E0F3
:109E10000E947F4B8091970790919807892B71F052
:109E20008091740990917509019741F40E94430E45
:109E3000AB01BC0181E00E940B4C1DC088E061E0D9
:109E400046E753E10E94B41916C00630A1F48CE035
:109E50000E948C4B85E061E041E653E10E94B41919
:109E60000E94994B08C00E945E0EAB01BC0180E0CD
:109E70000E940B4CCCCF6096E8E00C94B56180E07A
:109E800091E0EDE7FAE0DF019C011D9221503040A6
:109E9000E1F7089580E091E0EDE7F9E0DF019C0152
:109EA0001D9221503040E1F70895EF92FF920F93F9
:109EB0001F93182F8DE89AE06DE77AE040EF50E0AD
:109EC0000E9437626091270170912801E09125017D
:109ED000E0902301F090210100911F01F0911D01FC
:109EE000153079F44091120450911304209110041C
:109EF0003091110480910E0490910F04A0E0B0E025
:109F000032C01A3011F0173089F48091B904482F0B
:109F100050E08091BA04282F30E08091BB049091EA
:109F2000BC04A091BD04B091BE041DC0812F885017
:109F3000823048F080E090E0A0E0B0E020E030E047
:109F400040E050E010C040912B0450912C0420912F
:109F5000290430912A048091210490912204A09137
:109F60002304B09124048093890A90938A0AA093D1
:109F70008B0AB0938C0A3093880A2093870A5093F7
:109F8000860A4093850A1093840AF093830A00930B
:109F9000820AF092810AE092800AEF5FE0937F0AE2
:109FA0006459784F70937E0A60937D0A1A3079F075
:109FB0001B3169F0113259F01C3049F01D3039F075
:109FC000113029F0123019F0143009F017981F9150
:109FD0000F91FF90EF900895FF920F931F93F82E2B
:109FE0008DE899E08C0100511040B80140EF50E03D
:109FF0000E94376280912701909128018459984FDF
:10A00000509125015F5FB0912301A0912101F09152
:10A010001F01E0911D0160917307709174072091F9
:10A020007507309176074091720710928C09109253
:10A030008B0910928A0940938909F0928409309320
:10A040008809209387097093860960938509E093B6
:10A050008309F0938209A0938109B09380095093FA
:10A060007F09F801918380831F910F91FF900895DC
:10A070001F93CF93DF93EC01162F1092910B1E8646
:10A080000C960E94A53C8E3391050CF066C090930F
:10A090006601809365011C86CE010A960E94A53C4C
:10A0A0008C3391050CF059C090936801809367013F
:10A0B0001A86CE0108960E94A53C883191050CF0C5
:10A0C0004CC090936A01809369011886CE01069670
:10A0D0000E94A53C009709F440C080329105ECF540
:10A0E00090936C0180936B011E82CE0104960E94B6
:10A0F000A53C01978C30910584F590936E01809377
:10A100006D011C82CE010E94A53C8C569740909315
:10A11000700180936F011092720110927101109280
:10A1200074011092730185E691E00E94441D6093D2
:10A130008B0B70938C0B80938D0B90938E0B809177
:10A140008B0B90918C0BA0918D0BB0918E0BB7FD6A
:10A1500002C01093910B81E001C080E0DF91CF91AC
:10A160001F910895AF92BF92CF92DF92EF92FF922C
:10A170000F931F93379B08C01092770910927609AE
:10A1800089E080937D017AC180917D01893019F445
:10A1900082E080937D0110917309112309F46EC14F
:10A1A0001130D9F41092910B0E94961A8091760981
:10A1B00090917709892B19F483EA93E102C08CE925
:10A1C00093E10E94BF1B82E0809373090E945C1A96
:10A1D000909379098093780951C11230D9F50E9482
:10A1E000AA1A813009F034C18091760990917709DB
:10A1F000892BC1F488E893E066E973E145E050E01B
:10A200000E940662892B39F481E090E090937709EF
:10A210008093760911C080E490E00E947B0E109339
:10A220007D0113C188E893E06DE873E148E050E0F8
:10A230000E940662892B11F483E052C0A1E4B1E0D0
:10A24000EDE1F1E082E101900D928150E1F7109291
:10A25000730915C1133041F40E94961A86E893E100
:10A260000E94BF1B84E0B0CF143009F051C00E949F
:10A27000AA1A813009F03FC01092920380E993E05E
:10A280000E94A53C009779F18032910564F5909386
:10A290006C0180936B0110928F038DE893E00E9414
:10A2A000A53C01978C309105F4F490936E01809356
:10A2B0006D0110928C0388E893E00E94A53C8C56B7
:10A2C000974097FD10C09093700180936F0110929A
:10A2D000720110927101109274011092730185E065
:10A2E00080937309CBC080E490E00E947B0E81E0F4
:10A2F00080937D01AAC00E945C1A20917809309158
:10A300007909821B930B805D974008F4B7C0ABC0FE
:10A31000153041F40E94961A8FE793E10E94BF1B0B
:10A3200086E052CF163009F0A9C00E94AA1A8130E7
:10A3300009F08EC0109290038EE893E00E94A53C35
:10A340008C3391050CF081C0909366018093650178
:10A3500010928D038BE893E00E94A53C8C3391050D
:10A360000CF073C0909368018093670110928A0388
:10A3700088E893E00E94A53C883191050CF065C007
:10A3800090936A018093690185E691E00E94441DE3
:10A390007B018C0180E7A82E81E8B82E8FEFC82EB4
:10A3A0008FEFD82EEA0CFB1C0C1D1D1D17FD48C09D
:10A3B000F89420917F0B3091800B4091810B50914C
:10A3C000820B789480911B0190911C01892B01F5DF
:10A3D00080919C0790919D070097D1F057016801EB
:10A3E000A21AB30AC40AD50AA6019501D7FE07C06E
:10A3F00050954095309521953F4F4F4F5F4FA0E0CE
:10A40000B0E082179307A407B50714F482E019C0DF
:10A41000E0928B0BF0928C0B00938D0B10938E0BB4
:10A4200081E08093910B109276071092750710923D
:10A4300074071092730710927D0110927C0105C081
:10A4400081E080937D010E946F0B1092730916C00A
:10A450000E945C1A2091780930917909821B930B34
:10A46000805D974058F080E490E00E947B0E83E08E
:10A4700080937D011092730985E201C080E01F91F5
:10A480000F91FF90EF90DF90CF90BF90AF90089525
:10A49000A1E0B0E0EEE4F2E50C949561182F0E9483
:10A4A000961A183019F48FE094E106C0103111F0BB
:10A4B000CC244BC08BED93E10E94BF1B0E945C1A21
:10A4C0005C018C01CC24DD244E010894811C911C7C
:10A4D00002C0DD2487010E945C1A7C01081719075D
:10A4E00009F0A895C7018A199B09805D974018F06B
:10A4F00025E2C22E2AC0DD2059F4C4010E94791A37
:10A50000813041F78981843229F7DD24D394E2CF69
:10A5100081E0D81669F40E94AA1AC82E21E0821799
:10A5200019F492E0D92ED6CF82E0C81699F60DC064
:10A5300022E0D21679F688E893E06DEC73E14DE005
:10A5400050E00E940662892B21F68C2D2196ECE0CA
:10A550000C94B161A0E1B0E0E0EBF2E50C949C61F9
:10A5600088E893E06CE270E00E945B62009709F477
:10A570009DC08C010F5F1F4FCE010996B80146E0C8
:10A5800050E00E948462C8016CE270E00E945B624D
:10A59000FC01009709F48AC0F18001966CE270E03A
:10A5A0000E945B62009709F481C001966CE270E042
:10A5B0000E945B62009709F479C001966CE270E03A
:10A5C0000E945B62009709F471C001966CE270E032
:10A5D0000E945B62009709F469C001966CE270E02A
:10A5E0000E945B62009709F461C001966CE270E022
:10A5F0000E945B62009709F459C001966CE270E01A
:10A600000E945B628C01009709F450C0BC016F5F2F
:10A610007F4FCE01079642E050E00E948462B8016D
:10A620006D5F7F4FCE01059642E050E00E9484624C
:10A63000B8016B5F7F4FCE01039642E050E00E946D
:10A640008462F8018581873324F081E3898389E37B
:10A6500003C082E3898380E38A83CE01019661E0AF
:10A6600070E00E943850882311F482E220C0F1E4A7
:10A67000FF1661F48091900B882311F087E001C0F0
:10A6800086E080937D0110927C010EC086E5F8166D
:10A6900069F488E080937D01809167099091680951
:10A6A000892B89F30E946F0B80E001C083E26096E2
:10A6B000E5E00C94B861A0E1B0E0E1E6F3E50C94CC
:10A6C0009B6188E080937D0188E893E06CE270E014
:10A6D0000E945B62009791F08C010F5F1F4FCE01CB
:10A6E0000996B80146E050E00E948462C8016CE21D
:10A6F00070E00E945B627C01009721F40E946F0B66
:10A7000083E239C00894E11CF11CCE010796B70121
:10A7100042E050E00E94846283E090E0E80EF91E7F
:10A72000CE010596B70142E050E00E94846283E0CA
:10A7300090E0E80EF91E8E010F5F1F4FC801B701B0
:10A7400044E050E00E948462C80161E070E00E9431
:10A750003850882321F40E946F0B82E20CC0809154
:10A76000900B882311F087E001C086E080937D0183
:10A7700010927C0180E06096E6E00C94B761FC01E9
:10A78000808191819A3239F09A3029F0319699235B
:10A7900011F08927F6CF0E94543B0895A5E0B0E060
:10A7A000E4EDF3E50C949E6180910B0490910C0410
:10A7B000892BD1F4CE0101960E94791A813009F0DB
:10A7C000F1C08981843209F0EDC00E945C1A909337
:10A7D0000A048093090481E090E090930C04809334
:10A7E0000B0410920804DEC00E94AA1A813009F0FE
:10A7F000C8C010916409187309F069C088E893E033
:10A8000062EC73E14AE050E00E940662892B09F095
:10A81000C9C090919303993331F481E380939103FC
:10A820009093920306C082E38093910380E3809328
:10A83000920381E993E062E070E00E943850813039
:10A8400011F082E2B2C0F89410927E0B10927D0B50
:10A8500080918B0B90918C0BA0918D0BB0918E0BF6
:10A8600080938B0790938C07A0938D07B0938E07EE
:10A8700080937F0B9093800BA093810BB093820BFE
:10A8800078948091A003813311F484E00EC0823368
:10A8900021F485E080937D0117C0833309F082C0E5
:10A8A0008091A203803351F486E080937D018091F2
:10A8B000670990916809892B39F403C087E0809378
:10A8C0007D0110927C016EC00E946F0B6BC088E806
:10A8D00093E0BE016E5F7F4F0E94BF5388E893E014
:10A8E0006AE270E00E945B62FC0191818A819817A4
:10A8F00009F05AC092818B81981709F055C088E8F9
:10A9000093E066E971E044E050E00E9476620097CF
:10A9100031F48091640980688093640943C01830E1
:10A92000B9F488E893E06CEB73E145E050E00E94F5
:10A930000662892B51F088E893E066EB73E145E00D
:10A9400050E00E940662892B69F50E94AA522DC030
:10A95000103141F588E893E060EB73E145E050E0A9
:10A960000E940662892B51F088E893E06AEA73E15D
:10A9700045E050E00E940662892BA1F40E945B53DF
:10A9800014C00E945C1A2091090430910A04821BB1
:10A99000930B885E934030F010920C0410920B04DD
:10A9A00085E203C080E001C084E22596E3E00C94D8
:10A9B000BA61A8E0B0E0EFEDF4E50C949B6181E0B2
:10A9C0000E94AE1981E061E044E656E10E94B419AC
:10A9D00080916709909168097E010894E11CF11C3F
:10A9E000B7010E94003CAC0186E061E00E94C419FE
:10A9F00086E061E0A70125E000E010E00E941F3F33
:10AA0000892B19F421E030E012C0C7010E94A53C57
:10AA1000BC01909368098093670901C0A895F999D2
:10AA2000FDCF82ED90E00E94DD6220E030E0C901C0
:10AA30002896E6E00C94B761A8E0B0E0E2E2F5E524
:10AA40000C949B6181E00E94AE1981E061E042E7D5
:10AA500056E10E94B41980916509909166097E01C2
:10AA60000894E11CF11CB7010E94003CAC0186E097
:10AA700061E00E94C41986E061E0A70125E000E0E2
:10AA800010E00E941F3F892B19F421E030E012C032
:10AA9000C7010E94A53CBC0190936609809365099B
:10AAA00001C0A895F999FDCF80ED90E00E94DD628C
:10AAB00020E030E0C9012896E6E00C94B7611F93CE
:10AAC000182F0E948319E12FF0E0EE0FFF1FEC5CBE
:10AAD000FA4E4591549180E060E00E94B4191F91B4
:10AAE0000895A8E0B0E0E7E7F5E50C949B618EE0FF
:10AAF0000E945F5581E061E045E456E10E94B4198F
:10AB000080919C0790919D077E010894E11CF11CA7
:10AB1000B7010E94003CAC0187E061E00E94C419CB
:10AB200087E061E0A70125E000E010E00E941F3F00
:10AB3000892B19F421E030E012C0C7010E94A53C26
:10AB4000BC0190939D0780939C0701C0A895F9993B
:10AB5000FDCF88EC90E00E94DD6220E030E0C9018A
:10AB60002896E6E00C94B761A8E0B0E0EAEBF5E5E2
:10AB70000C949B618DE00E945F5581E061E044E5AB
:10AB800056E10E94B41980919507909196077E0135
:10AB90000894E11CF11CB7010E94003CAC0189E063
:10ABA00061E00E94C41989E061E0A70125E000E0AE
:10ABB00010E00E941F3F892B19F421E030E012C001
:10ABC000C7010E94A53CBC0190939607809395070E
:10ABD00001C0A895F999FDCF86EC90E00E94DD6256
:10ABE00020E030E0C9012896E6E00C94B761EF92CE
:10ABF000FF921F93DF93CF930F92CDB7DEB78CE018
:10AC00000E945F558091640990E036E096958795A3
:10AC10003A95E1F7182F1170E12FF0E0EE0FFF1FCA
:10AC2000EF5EF94E4591549180E061E00E94B419C5
:10AC30007E010894E11CF11C812F62E0A7010E94B3
:10AC4000FC3E182F89818931A1F1843111F501C0B1
:10AC5000A895F999FDCF8CE390E00E94A96220911C
:10AC60006409112331F42F7B20936409BC01677FB1
:10AC700007C0206420936409BC01686001C0A895E6
:10AC8000F999FDCF8CE390E00E94DD6220E030E096
:10AC900012C081E00E94AE19E12FF0E0EE0FFF1F1D
:10ACA000EF5EF94E4591549180E061E00E94B41945
:10ACB000C3CF21E030E0C9010F90CF91DF911F9108
:10ACC000FF90EF900895EF92FF921F93DF93CF9341
:10ACD0000F92CDB7DEB78BE00E945F5510916409EB
:10ACE0001695169516951770E12FF0E0EE0FFF1FE1
:10ACF000E950FA4E4591549180E061E00E94B41908
:10AD00007E010894E11CF11C812F63E0A7010E94E1
:10AD1000FC3E182F8981893109F43AC0843141F50C
:10AD200001C0A895F999FDCF8CE390E00E94A9623B
:10AD3000BC01687F80916409877C112319F480939A
:10AD400064090DC0113029F4886080936409616042
:10AD500006C0806180936409626001C0A895F9997A
:10AD6000FDCF8CE390E00E94DD6220E030E012C075
:10AD700081E00E94AE19E12FF0E0EE0FFF1FE950D5
:10AD8000FA4E4591549180E061E00E94B419BCCF25
:10AD900021E030E0C9010F90CF91DF911F91FF902A
:10ADA000EF900895CF92DF92FF920F931F93DF935E
:10ADB000CF930F92CDB7DEB788E00E945F55F09039
:10ADC0007209EF2DF0E0EE0FFF1FE855FA4E4591A6
:10ADD000549180E061E00E94B4196E010894C11C96
:10ADE000D11C8F2D66E0A6010E94FC3EF82E8981C1
:10ADF000893109F434C00F2D10E0843109F5F09247
:10AE00007209F801EE0FFF1FEE0FFF1FEC54FA4E10
:10AE100085919591A591B491809377019093780154
:10AE2000A0937901B0937A0101C0A895F999FDCF5B
:10AE30008CEC90E0B8010E94DD6220E030E011C0AF
:10AE400081E00E94AE19F801EE0FFF1FE855FA4E9F
:10AE50004591549180E061E00E94B419C2CF21E095
:10AE600030E0C9010F90CF91DF911F910F91FF90BA
:10AE7000DF90CF900895CF92DF92FF920F931F93B0
:10AE8000DF93CF930F92CDB7DEB787E00E945F5577
:10AE900001C0A895F999FDCF8AEC90E00E94A962C3
:10AEA0008C01FF24F394F822EF2DF0E0EE0FFF1F4A
:10AEB000EF5BF94E4591549180E061E00E94B41936
:10AEC0006E010894C11CD11C8F2D62E0A6010E9466
:10AED000FC3EF82E8981893191F1843101F5809110
:10AEE0006409982F9770FF2031F4B8016E7F91307C
:10AEF00061F4887F06C0B8016160992331F4887FCE
:10AF000081608093640901C0A895F999FDCF7F778E
:10AF10008AEC90E00E94DD6220E030E012C081E027
:10AF20000E94AE19EF2DF0E0EE0FFF1FEF5BF94E20
:10AF30004591549180E061E00E94B419C5CF21E0B1
:10AF400030E0C9010F90CF91DF911F910F91FF90D9
:10AF5000DF90CF900895A8E0B0E0E1EBF7E50C9426
:10AF60009B6186E00E945F5580E061E040E856E129
:10AF70000E94B41980919707909198077E010894D8
:10AF8000E11CF11CB7010E94003CAC0189E061E0CA
:10AF90000E94C41989E061E0A70125E000E010E00B
:10AFA0000E941F3F892B19F421E030E012C0C70135
:10AFB0000E94A53CBC01909398078093970701C01D
:10AFC000A895F999FDCF84EC90E00E94DD6220E025
:10AFD00030E0C9012896E6E00C94B761A4E1B0E046
:10AFE000E4EFF7E50C9499616B010E945F5501C095
:10AFF000A895F999FDCFC6010E94A36269837A835F
:10B000008B839C8325E0E22EF12CEC0EFD1EA70124
:10B010000E94523E81E061E0A7012FE000E010E0D5
:10B020000E941F3F892B19F421E030E015C0C701B1
:10B03000BE016F5F7F4F0E94EE3D813059F401C029
:10B04000A895F999FDCF49815A816B817C81C60110
:10B050000E94D16220E030E0C9016496E8E00C94DF
:10B06000B56185E060EC70E00E94EE57089583E0E2
:10B070006CE270E00E94EE57089582E068E270E0B2
:10B080000E94EE57089581E064E270E00E94EE575E
:10B09000089580E060E270E00E94EE570895CF923C
:10B0A000DF92FF920F931F93DF93CF930F92CDB751
:10B0B000DEB784E00E945F5501C0A895F999FDCFE5
:10B0C0008CE090E00E94A9628C01F12EFF1CFF240D
:10B0D000FF1CEF2DF0E0EE0FFF1FEC5DF94E4591E8
:10B0E000549180E061E00E94B4196E010894C11C83
:10B0F000D11C8F2D62E0A6010E94FC3EF82E8981B2
:10B10000893141F18431B1F4FF2029F41092D5073F
:10B11000B8017F7706C08093D507B801706801C079
:10B12000A895F999FDCF8CE090E00E94DD6220E0C7
:10B1300030E012C081E00E94AE19EF2DF0E0EE0F7A
:10B14000FF1FEC5DF94E4591549180E061E00E9453
:10B15000B419CFCF21E030E0C9010F90CF91DF913A
:10B160001F910F91FF90DF90CF900895A4E0B0E081
:10B17000ECEBF8E50C949E61182F0E94831980E097
:10B1800060E044E956E10E94B419E12FFF27E7FD92
:10B19000F095EE0FFF1FEC5CFA4E4591549180E064
:10B1A00061E00E94B419812F8F5FBE016F5F7F4FF6
:10B1B0000E94E43B8BE060E0AE014E5F5F4F0E9477
:10B1C000C4198DE060E040E956E10E94B41924966C
:10B1D000E3E00C94BA61CF92DF92FF920F931F933A
:10B1E000DF93CF93CDB7DEB76F970FB6F894DEBF7E
:10B1F0000FBECDBFDE011296EBE9F1E08EE10190CA
:10B200000D928150E1F70E94B658FF246E01089418
:10B21000C11CD11C8F2D60E1A6010E94FC3EF82EBE
:10B2200089818931C1F0843119F000E010E00EC04D
:10B230008FE0F81681F0EF2DF0E0EE0FFF1FEC0D20
:10B24000FD1D0180F281E02D09958C018F2D0E945A
:10B25000B658012BF9F28091D507882309F045C033
:10B260001092D7071092D60780E290E044E651E0B2
:10B2700068EA70EC0E94981B6093AA047093AB0478
:10B280008093AC049093AD0484E290E040E05FEFE3
:10B290006FEF7FEF0E94981B6093AE047093AF0432
:10B2A0008093B0049093B10488E290E041E051E0D3
:10B2B00068EA70EC0E94981B6093B2047093B30428
:10B2C0008093B4049093B5048CE290E041E051E0A7
:10B2D00068EA70EC0E94981B60935E0970935F09A6
:10B2E000809360099093610917C08431A9F481E0CB
:10B2F00090E09093D7078093D607A8E0B1E0EDE106
:10B30000F1E082E101900D928150E1F70E94BD27AA
:10B31000882311F00E94554F6F960FB6F894DEBF48
:10B320000FBECDBFCF91DF911F910F91FF90DF90A6
:10B33000CF900895EF92FF920F93DF93CF93CDB705
:10B34000DEB760970FB6F894DEBF0FBECDBFA82F53
:10B35000002309F461C07E010894E11CF11C88E01F
:10B36000F70111928A95E9F729833A834B835C832D
:10B370006D837E83AF83988780E2801BE82FFF2751
:10B38000E7FDF09549815A816B817C81181684F024
:10B3900019861A861B861C86882799278E1B9F0B69
:10B3A00004C0440F551F661F771F8A95D2F728C027
:10B3B000202F332727FD3095DB01CA01022E04C060
:10B3C000880F991FAA1FBB1F0A94D2F789879A87F3
:10B3D000AB87BC8704C07695679557954795EA95E6
:10B3E000D2F78D819E81AF81B88504C0880F991FE7
:10B3F000AA1FBB1F2A95D2F7482B592B6A2B7B2BF0
:10B400004D875E876F87788B29853A854B855C856C
:10B410006D857E85AF8598898A2F60960FB6F894E2
:10B42000DEBF0FBECDBFCF91DF910F91FF90EF90A8
:10B430000895EF92FF920F93DF93CF93CDB7DEB7CE
:10B4400060970FB6F894DEBF0FBECDBFA82F0023C4
:10B4500009F467C07E010894E11CF11C88E0F70143
:10B4600011928A95E9F729833A834B835C836D8334
:10B470007E83AF83988780E2801B4D815E816F81E0
:10B480007885E82FFF27E7FDF0951816B4F0DB016B
:10B49000CA01BB0F880B982FDC018D879E87AF8771
:10B4A000B88B882799278E1B9F0B04C075956795CD
:10B4B000579547958A95D2F728C0202F332727FD27
:10B4C0003095DB01CA01022E04C0B595A79597956A
:10B4D00087950A94D2F78D879E87AF87B88B04C073
:10B4E000440F551F661F771FEA95D2F789819A810D
:10B4F000AB81BC8104C0B695A795979587952A9591
:10B50000D2F7482B592B6A2B7B2B49875A876B879D
:10B510007C8729853A854B855C856D857E85AF85E1
:10B5200098898A2F60960FB6F894DEBF0FBECDBF04
:10B53000CF91DF910F91FF90EF900895AEE5B0E0CD
:10B54000E4EAFAE50C948F61A8E04E010894811CAE
:10B55000911CF4016A2E11926A94E9F729833A83C7
:10B560004B835C836D837E838F839887CE0109969E
:10B57000FC011192AA95E9F7A986BA86CB86DC86EA
:10B58000ED86FE860F87188B29843A844B845C8471
:10B59000ED84FE840F85188969807A808B809C8079
:10B5A0006DA67EA68FA698AA6D807E808F809884D7
:10B5B000E114F1040105110509F0B3C36214730429
:10B5C0008404950408F03DC100E0201600E0300638
:10B5D00001E0400600E0500688F41FEF2116310418
:10B5E0004104510439F030F048E0E42EF12C012DF3
:10B5F000112D18C0EE24FF24870114C020E022166C
:10B6000020E0320620E0420621E0520630F038E128
:10B61000E32EF12C012D112D05C020E1E22EF12C9D
:10B62000012D112DD201C1010E2C04C0B695A79594
:10B63000979587950A94D2F787549E4FDC012C91F9
:10B6400080E290E0A0E0B0E08E199F09A00BB10B62
:10B650007C018D01E21AF10801091109E114F104DC
:10B6600001051105A1F10E2C04C0220C331C441C51
:10B67000551C0A94D2F7A40193010E2C04C0220F8A
:10B68000331F441F551F0A94D2F780E290E08E19B1
:10B690009F096DA47EA48FA498A804C09694879453
:10B6A000779467948A95D2F7622A732A842A952A16
:10B6B000ADA4BEA4CFA4D8A804C0AA0CBB1CCC1CAB
:10B6C000DD1CEA94D2F7ADA6BEA6CFA6D8AA620129
:10B6D000EE24FF24CDAADEAAEFAAF8AE92018101E2
:10B6E0002070307009AF1AAF2BAF3CAFC401B3016B
:10B6F000A70196010E9452617B018C01C401B30134
:10B700002DA93EA94FA958AD0E945261C901DA0185
:10B710003C014D01C401B30129AD3AAD4BAD5CAD67
:10B720000E9413619B01AC018701FF24EE24ADA4AC
:10B73000BEA4CFA4D8A8C601AA27BB275701680179
:10B74000A82AB92ACA2ADB2AA216B306C406D50635
:10B75000E0F408946108710881089108A20CB31CF8
:10B76000C41CD51CA214B304C404D50470F0A216E2
:10B77000B306C406D50648F4089461087108810828
:10B780009108A20CB31CC41CD51CA21AB30AC40A8B
:10B79000D50AC601B5012DA93EA94FA958AD0E94F1
:10B7A00052617B018C01C601B5012DA93EA94FA9AB
:10B7B00058AD0E945261C901DA015C016D01C601F8
:10B7C000B50129AD3AAD4BAD5CAD0E9413619B0153
:10B7D000AC018701FF24EE248DA59EA5AFA5B8A9D5
:10B7E000A070B070E82AF92A0A2B1B2BE216F30688
:10B7F00004071507C0F40894A108B108C108D108CE
:10B80000E20CF31C041D151DE214F30404051505D8
:10B8100050F0E216F3060407150728F40894A1086F
:10B82000B108C108D108D30199278827860175017D
:10B83000E82AF92A0A2B1B2BE9AAFAAA0BAB1CABA4
:10B84000CFC4211431044104510471F461E070E06B
:10B8500080E090E020E030E040E050E00E94526163
:10B86000C901DA011C012D0100E0201600E03006BC
:10B8700001E0400600E0500688F41FEF2116310475
:10B880004104510431F028F048E050E060E070E0FD
:10B8900017C040E050E060E070E012C020E02216E7
:10B8A00020E0320620E0420621E0520628F048E17E
:10B8B00050E060E070E004C040E150E060E070E023
:10B8C000D201C101042E04C0B695A795979587951E
:10B8D0000A94D2F787549E4FDC012C91E0E2EE2EC1
:10B8E000F12C012D112DD801C701841B950BA60B3E
:10B8F000B70B821B9109A109B1090097A105B105F8
:10B9000061F464015301A218B308C408D50831E0FA
:10B91000632E712C812C912C1EC16F968FAF6F9767
:10B92000082E04C0220C331C441C551C0A94D2F768
:10B93000EE2DE81B640153010E2E04C0D694C7946B
:10B94000B794A7940A94D2F7A40193016F960FAC11
:10B950006F9704C0220F331F441F551F0A94D2F75C
:10B960006DA47EA48FA498A80E2E04C096948794EC
:10B97000779467940A94D2F784017301E22AF32A38
:10B98000042B152BE9A6FAA60BA71CA732018824C5
:10B990009924920181012070307021960CAF1DAF67
:10B9A0002EAF3FAF2197C601B501A40193010E94BC
:10B9B00052617B018C01C601B501A40193010E9473
:10B9C0005261C901DA0125968CAF9DAFAEAFBFAF12
:10B9D0002597BC01CD0121962CAD3DAD4EAD5FAD9F
:10B9E00021970E9413619B01AC018701FF24EE2483
:10B9F000A9A4BAA4CBA4DCA4C601AA27BB275C01D6
:10BA00006D01AE28BF28C02AD12AA216B306C406EB
:10BA1000D50660F525966CAD7DAD8EAD9FAD2597B5
:10BA2000615070408040904025966CAF7DAF8EAFE6
:10BA30009FAF2597A20CB31CC41CD51CA214B30441
:10BA4000C404D50498F0A216B306C406D50670F453
:10BA5000615070408040904025966CAF7DAF8EAFB6
:10BA60009FAF2597A20CB31CC41CD51CA21AB30A05
:10BA7000C40AD50AC601B501A40193010E9452610E
:10BA80007B018C01C601B501A40193010E945261A2
:10BA9000C901DA013C014D01C401B30121962CAD6D
:10BAA0003DAD4EAD5FAD21970E9413619B01AC018E
:10BAB0008701FF24EE2489A59AA5ABA5BCA5A0709B
:10BAC000B07057016801A82AB92ACA2ADB2AA2162F
:10BAD000B306C406D506E0F408946108710881082D
:10BAE0009108A20CB31CC41CD51CA214B304C4043A
:10BAF000D50470F0A216B306C406D50648F408941F
:10BB00006108710881089108A20CB31CC41CD51CE3
:10BB10008DA59EA5AFA5B8A96F960FAC6F9704C071
:10BB2000880F991FAA1FBB1F0A94D2F78DA79EA743
:10BB3000AFA7B8ABA21AB30AC40AD50A2596ECACD3
:10BB4000FDAC0EAD1FAD2597D70199278827682A30
:10BB5000792A8A2A9B2A82012227332729960CAF29
:10BB60001DAF2EAF3FAF2997A201910140705070D9
:10BB70002D962CAF3DAF4EAF5FAF2D97C601B501EF
:10BB800029962CAD3DAD4EAD5FAD29970E94526117
:10BB90007B018C01C601B50129962CAD3DAD4EADA2
:10BBA0005FAD29970E945261C901DA0161968CAF9D
:10BBB0009DAFAEAFBFAF6197BC01CD012D962CAD4F
:10BBC0003DAD4EAD5FAD2D970E9413619B01AC0161
:10BBD0008701FF24EE24ADA4BEA4CFA4D8A8C6013B
:10BBE000AA27BB2757016801A82AB92ACA2ADB2A33
:10BBF000A216B306C406D50660F561966CAD7DADA0
:10BC00008EAD9FAD619761507040804090406196CD
:10BC10006CAF7DAF8EAF9FAF6197A20CB31CC41CFD
:10BC2000D51CA214B304C404D50498F0A216B3061C
:10BC3000C406D50670F46150704080409040619613
:10BC40006CAF7DAF8EAF9FAF6197A20CB31CC41CCD
:10BC5000D51CA21AB30AC40AD50AC601B501299691
:10BC60002CAD3DAD4EAD5FAD29970E9452617B0179
:10BC70008C01C601B50129962CAD3DAD4EAD5FAD31
:10BC800029970E945261C901DA015C016D01C60168
:10BC9000B5012D962CAD3DAD4EAD5FAD2D970E94FB
:10BCA00013619B01AC018701FF24EE248DA59EA5A5
:10BCB000AFA5B8A9A070B070E82AF92A0A2B1B2BEF
:10BCC000E216F30604071507C0F40894A108B108AA
:10BCD000C108D108E20CF31C041D151DE214F30485
:10BCE0000405150550F0E216F3060407150728F4BD
:10BCF0000894A108B108C108D1086196ECACFDAC6C
:10BD00000EAD1FAD6197D701992788279601850150
:10BD1000082B192B2A2B3B2B09AB1AAB2BAB3CABBB
:10BD200062C26E147F048006910608F451C220E0BE
:10BD3000E21620E0F20621E0020720E0120788F474
:10BD40003FEFE316F1040105110531F028F048E05A
:10BD500050E060E070E017C040E050E060E070E06C
:10BD600012C040E0E41640E0F40640E0040741E081
:10BD7000140728F048E150E060E070E004C040E1C2
:10BD800050E060E070E0D801C701042E04C0B69511
:10BD9000A795979587950A94D2F787549E4FDC0113
:10BDA0002C9130E2A32EB12CC12CD12CD601C5018F
:10BDB000841B950BA60BB70B821B9109A109B10936
:10BDC0000097A105B10589F4E614F70408051905E3
:10BDD00008F4F2C16DA47EA48FA498A86214730421
:10BDE0008404950408F0E8C1F3C16E968FAF6E9796
:10BDF000082E04C0EE0CFF1C001F111F0A94D2F77E
:10BE00006A2D681BD201C101062E04C0B695A79504
:10BE1000979587950A94D2F75C016D01AE28BF28EB
:10BE2000C02AD12AADA2BEA2CFA2D8A672016101BA
:10BE30006E960FAC6E9704C0CC0CDD1CEE1CFF1C84
:10BE40000A94D2F7C9A2DAA2EBA2FCA264015301C0
:10BE5000062E04C0D694C794B794A7940A94D2F738
:10BE6000D401C3016E960FAC6E9704C0880F991F62
:10BE7000AA1FBB1F0A94D2F7EDA4FEA40FA518A910
:10BE800004C016950795F794E7946A95D2F73701A1
:10BE90004801682A792A8A2A9B2A6D8E7E8E8F8E87
:10BEA00098A2EDA0FEA00FA118A53801882499241E
:10BEB000980187012070307065960CAF1DAF2EAFD2
:10BEC0003FAF6597C601B501A40193010E9452617D
:10BED0007B018C01C601B501A40193010E9452614E
:10BEE000C901DA011C012D01C201B10165962CAD19
:10BEF0003DAD4EAD5FAD65970E9413619B01AC01F6
:10BF00008701FF24EE24AD8CBE8CCF8CD8A0C60157
:10BF1000AA27BB2757016801A82AB92ACA2ADB2AFF
:10BF2000A216B306C406D50600F508942108310808
:10BF300041085108EDA0FEA00FA118A5AE0CBF1C32
:10BF4000C01ED11EAE14BF04C006D10670F0A216EA
:10BF5000B306C406D50648F4089421083108410800
:10BF60005108AE0CBF1CC01ED11EA21AB30AC40ACF
:10BF7000D50AC601B501A40193010E9452617B015B
:10BF80008C01C601B501A40193010E945261C9014F
:10BF9000DA013C014D01C401B30165962CAD3DAD04
:10BFA0004EAD5FAD65970E9413619B01AC018701A7
:10BFB000FF24EE248D8D9E8DAF8DB8A1A070B07042
:10BFC00057016801A82AB92ACA2ADB2AA216B30691
:10BFD000C406D50600F50894610871088108910827
:10BFE0006DA17EA18FA198A5A60EB71EC81ED91E51
:10BFF000A616B706C806D90670F0A216B306C40680
:10C00000D50648F408946108710881089108A60EC5
:10C01000B71EC81ED91ED601C501821B930BA40BE7
:10C02000B50B898F9A8FAB8FBC8FD1019927882749
:10C0300064015301A82AB92ACA2ADB2AA9AABAAAE2
:10C04000CBAADCAA860175012FEF3FEF40E050E05C
:10C05000E222F32204231523A601662777276D9693
:10C060004CAF5DAF6EAF7FAF6D97A9A0BAA0CBA06C
:10C07000DCA06FEF7FEF80E090E0A622B722C8221D
:10C08000D92289A19AA1ABA1BCA11D0144245524A8
:10C09000C801B701A60195010E94136169966CAFB2
:10C0A0007DAF8EAF9FAF6997C801B701A201910123
:10C0B0000E9413613B014C016D966CAD7DAD8EAD60
:10C0C0009FAD6D97A60195010E9413617B018C01C4
:10C0D0006D966CAD7DAD8EAD9FAD6D97A20191015A
:10C0E0000E9413615B016C01A8019701260D371DA9
:10C0F000481D591D69966CAC7DAC8EAC9FAC6997A0
:10C10000C401AA27BB27280F391F4A1F5B1F2E1502
:10C110003F054007510748F4E12CF12C61E0062F60
:10C12000112DAE0CBF1CC01ED11ECA01AA27BB27F1
:10C13000BC01CD016A0D7B1D8C1D9D1D698C7A8C07
:10C140008B8C9C8C661677068806990640F16615DE
:10C1500077058805990509F043C0D90199278827F3
:10C1600069962CAD3DAD4EAD5FAD69974070507096
:10C17000820F931FA41FB51F2DA53EA54FA558A93B
:10C180006E960FAC6E9704C0220F331F441F551FCD
:10C190000A94D2F7281739074A075B0708F509A957
:10C1A0001AA92BA93CA9015010402040304009ABEE
:10C1B0001AAB2BAB3CAB14C066247724430121E0BF
:10C1C00030E040E050E029AB3AAB4BAB5CAB0BC08E
:10C1D00066247724430119AA1AAA1BAA1CAA03C021
:10C1E000662477244301FE01719688E0DF011D92E9
:10C1F0008A95E9F7A9A8BAA8CBA8DCA8A98ABA8A1F
:10C20000CB8ADC8A6D8A7E8A8F8A988E29A93A89A0
:10C210004B895C89662D7E898F89988DC25ADF4F44
:10C22000E2E10C94AB61629FD001739FF001829FA9
:10C23000E00DF11D649FE00DF11D929FF00D839FB5
:10C24000F00D749FF00D659FF00D9927729FB00D52
:10C25000E11DF91F639FB00DE11DF91FBD01CF0165
:10C2600011240895991B79E004C0991F961708F0CE
:10C27000961B881F7A95C9F780950895AA1BBB1B4A
:10C2800051E107C0AA1FBB1FA617B70710F0A61BD6
:10C29000B70B881F991F5A95A9F780959095BC01F7
:10C2A000CD010895A1E21A2EAA1BBB1BFD010DC0F2
:10C2B000AA1FBB1FEE1FFF1FA217B307E407F50756
:10C2C00020F0A21BB30BE40BF50B661F771F881F32
:10C2D000991F1A9469F760957095809590959B01C8
:10C2E000AC01BD01CF01089597FB092E05260ED0A4
:10C2F00057FD04D0D7DF0AD0001C38F45095409584
:10C30000309521953F4F4F4F5F4F0895F6F7909529
:10C310008095709561957F4F8F4F9F4F08952F9215
:10C320003F924F925F926F927F928F929F92AF92C5
:10C33000BF92CF92DF92EF92FF920F931F93CF9312
:10C34000DF93CDB7DEB7CA1BDB0B0FB6F894DEBFA9
:10C350000FBECDBF09942A88398848885F846E84CF
:10C360007D848C849B84AA84B984C884DF80EE8019
:10C37000FD800C811B81AA81B981CE0FD11D0FB622
:10C38000F894DEBF0FBECDBFED010895911106C038
:10C3900080538A5010F0865C06C00895992788273C
:10C3A000089585FDFBCF80629111F8CF81568A51A7
:10C3B000E0F708959111089581568A5108F480524A
:10C3C00085580895FB01DC010D900020E9F71197D5
:10C3D00005900D920020E1F70895FB01DC018D919D
:10C3E000059080190110D9F3990B0895FB01DC0128
:10C3F00005900D920020E1F70895FC0105900020C2
:10C40000E9F7809590958E0F9F1F0895FB01DC0141
:10C410004150504030F08D910590801919F4002062
:10C42000B9F7881B990B0895FB0155915523A9F085
:10C43000BF01DC014D9145174111E1F759F4CD01E0
:10C440000590002049F04D9140154111C9F3FB01C1
:10C450004111EFCF81E090E001970895FB01DC01ED
:10C4600002C001900D9241505040D8F708956817CE
:10C47000790768F4FB01DC01E40FF51FA40FB51F79
:10C4800002C002900E9241505040D8F708950C948B
:10C490002E62DC0101C06D9341505040E0F70895D9
:10C4A000FB01DC010D900020E9F7119701900D923E
:10C4B0000020E1F70895FC018191861721F088237F
:10C4C000D9F7992708953197CF010895FB01DC0131
:10C4D0008D91019080190110D9F3990B0895FB01FA
:10C4E000DC0101900D920020E1F70895FB01DC01D1
:10C4F0004150504030F08D910190801919F4002086
:10C50000B9F7881B990B0895FB01DC01415050409D
:10C5100048F001900D920020C9F701C01D924150D2
:10C520005040E0F70895DC01CB01FC01F999FECF02
:10C5300006C0F2BDE1BDF89A319600B40D924150AB
:10C540005040B8F70895A6E1B0E044E050E00C9404
:10C550009562A8E1B0E042E050E00C949562DC0105
:10C56000A40FB51F4150504048F0CB01840F951FD8
:10C570002E910E94C06241505040D0F70895262F5E
:10C58000F999FECF92BD81BDF89A019700B40216C9
:10C5900039F01FBA20BD0FB6F894FA9AF99A0FBE77
:10C5A00008950396272F0E94C0620E94BF62252F24
:10C5B0000E94C062242F0C94C0620196272F0E9413
:10C5C000C0620C94BF62DC01CB0103C02D910E94BC
:10C5D000EE6241505040D0F70895262FF999FECFD2
:10C5E0001FBA92BD81BD20BD0FB6F894FA9AF99A90
:10C5F0000FBE01960895242F0E94EE62252F0E94FF
:10C60000EE620C9403630E94ED62272F0C94EE629D
:04C61000F894FFCFCC
:10C61400020000000000C01000000000090001003A
:10C6240000004600000000000000060100000000B9
:10C6340000090001000000460000000000000000A6
:10C64400000000000001000000460000000000009F
:10C654000000000000090001000000460000000086
:10C664000000000000000009000100000046000076
:10C674000000000000000000000900010000004666
:10C6840000000000000000907E0000C8040215CDE8
:10C694005B07E5559A15B53B121F33134905F1069F
:10C6A400110731075107504D544B00495843583D29
:10C6B4005837584F583158AB573B57D2561C55D959
:10C6C400546356F755B45571550001020203030330
:10C6D4000304040404040404040505050505050510
:10C6E40005050505050505050506060606060606EF
:10C6F40006060606060606060606060606060606D6
:10C7040006060606060606060607070707070707BE
:10C7140007070707070707070707070707070707A5
:10C724000707070707070707070707070707070795
:10C734000707070707070707070707070707070785
:10C74400070707070707070707080808080808086E
:10C754000808080808080808080808080808080855
:10C764000808080808080808080808080808080845
:10C774000808080808080808080808080808080835
:10C784000808080808080808080808080808080825
:10C794000808080808080808080808080808080815
:10C7A4000808080808080808080808080808080805
:10C7B40008080808080808080808080808080808F5
:0AC7C4000808080808080808080023
:00000001FF
